 NonConcreteKlassFilter

 Timestamp is 468608f0 (reproducible build file hash)

 Preferred load address is 0000000180000000

 Start         Length     Name                   Class
 0001:00000000 000038f0H .text$mn                CODE
 0001:000038f0 00000036H .text$mn$00             CODE
 0001:00003926 00000092H .text$x                 CODE
 0002:00000000 000001c8H .idata$5                DATA
 0002:000001c8 00000038H .00cfg                  DATA
 0002:00000200 00000008H .CRT$XCA                DATA
 0002:00000208 00000008H .CRT$XCZ                DATA
 0002:00000210 00000008H .CRT$XIA                DATA
 0002:00000218 00000008H .CRT$XIC                DATA
 0002:00000220 00000008H .CRT$XIZ                DATA
 0002:00000228 00000008H .CRT$XLA                DATA
 0002:00000230 00000008H .CRT$XLZ                DATA
 0002:00000238 00000008H .CRT$XPA                DATA
 0002:00000240 00000008H .CRT$XPZ                DATA
 0002:00000248 00000008H .CRT$XTA                DATA
 0002:00000250 00000010H .CRT$XTZ                DATA
 0002:00000258 00000000H .gehcont$y              DATA
 0002:00000258 00000000H .gfids$y                DATA
 0002:00000260 000023a0H .rdata                  DATA
 0002:00002600 00000000H .rdata$CastGuardVftablesA DATA
 0002:00002600 00000000H .rdata$CastGuardVftablesC DATA
 0002:00002600 00000028H .rdata$T                DATA
 0002:00002628 000000bcH .rdata$voltmd           DATA
 0002:000026e4 00000324H .rdata$zzzdbg           DATA
 0002:00002a08 00000008H .rtc$IAA                DATA
 0002:00002a10 00000008H .rtc$IZZ                DATA
 0002:00002a18 00000008H .rtc$TAA                DATA
 0002:00002a20 00000008H .rtc$TZZ                DATA
 0002:00002a28 00000004H .tls                    DATA
 0002:00002a2c 00000004H .tls$                   DATA
 0002:00002a30 00000008H .tls$ZZZ                DATA
 0002:00002a38 00000368H .xdata                  DATA
 0002:00002da0 00000370H .edata                  DATA
 0002:00003110 0000008cH .idata$2                DATA
 0002:0000319c 00000014H .idata$3                DATA
 0002:000031b0 000001c8H .idata$4                DATA
 0002:00003378 00000486H .idata$6                DATA
 0003:00000000 000000a0H .data                   DATA
 0003:000000a0 0001b238H .bss                    DATA
 0004:00000000 000003fcH .pdata                  DATA

  Address         Publics by Value              Rva+Base               Lib:Object

 0000:00000000       __AbsoluteZero             0000000000000000     <absolute>
 0000:00000000       ___safe_se_handler_count   0000000000000000     <absolute>
 0000:00000000       ___safe_se_handler_table   0000000000000000     <absolute>
 0000:00000000       __arm64x_extra_rfe_table   0000000000000000     <absolute>
 0000:00000000       __arm64x_extra_rfe_table_size 0000000000000000     <absolute>
 0000:00000000       __arm64x_native_entrypoint 0000000000000000     <absolute>
 0000:00000000       __arm64x_redirection_metadata 0000000000000000     <absolute>
 0000:00000000       __arm64x_redirection_metadata_count 0000000000000000     <absolute>
 0000:00000000       __dynamic_value_reloc_table 0000000000000000     <absolute>
 0000:00000000       __enclave_config           0000000000000000     <absolute>
 0000:00000000       __guard_check_icall_a64n_fptr 0000000000000000     <absolute>
 0000:00000000       __guard_eh_cont_count      0000000000000000     <absolute>
 0000:00000000       __guard_eh_cont_table      0000000000000000     <absolute>
 0000:00000000       __guard_fids_count         0000000000000000     <absolute>
 0000:00000000       __guard_fids_table         0000000000000000     <absolute>
 0000:00000000       __guard_iat_count          0000000000000000     <absolute>
 0000:00000000       __guard_iat_table          0000000000000000     <absolute>
 0000:00000000       __guard_longjmp_count      0000000000000000     <absolute>
 0000:00000000       __guard_longjmp_table      0000000000000000     <absolute>
 0000:00000000       __hybrid_auxiliary_iat     0000000000000000     <absolute>
 0000:00000000       __hybrid_auxiliary_iat_copy 0000000000000000     <absolute>
 0000:00000000       __hybrid_code_map          0000000000000000     <absolute>
 0000:00000000       __hybrid_code_map_count    0000000000000000     <absolute>
 0000:00000000       __x64_code_ranges_to_entry_points 0000000000000000     <absolute>
 0000:00000000       __x64_code_ranges_to_entry_points_count 0000000000000000     <absolute>
 0000:00000100       __guard_flags              0000000000000100     <absolute>
 0000:00000000       __ImageBase                0000000180000000     <linker-defined>
 0001:00000000       ?NewObject@JNIEnv_@@QEAAPEAV_jobject@@PEAV_jclass@@PEAU_jmethodID@@ZZ 0000000180001000 f i libNonConcreteKlassFilter.obj
 0001:00000028       ?SetEventNotificationMode@_jvmtiEnv@@QEAA?AW4jvmtiError@@W4jvmtiEventMode@@W4jvmtiEvent@@PEAV_jobject@@ZZ 0000000180001028 f i libNonConcreteKlassFilter.obj
 0001:00000034       ?TranslateError@@YAPEBDW4jvmtiError@@@Z 0000000180001034 f   libNonConcreteKlassFilter.obj
 0001:000002ec       ?nsk_jni_check_exception@@YAHPEAUJNIEnv_@@QEBDH@Z 00000001800012ec f   libNonConcreteKlassFilter.obj
 0001:00000430       ?nsk_jni_lverify@@YAHHPEAUJNIEnv_@@HQEBDH1ZZ 0000000180001430 f   libNonConcreteKlassFilter.obj
 0001:000004d0       Agent_Initialize           00000001800014d0 f   libNonConcreteKlassFilter.obj
 0001:000006e0       Agent_OnAttach             00000001800016e0 f   libNonConcreteKlassFilter.obj
 0001:000006e0       Agent_OnLoad               00000001800016e0 f   libNonConcreteKlassFilter.obj
 0001:000006e8       Java_nsk_jvmti_unit_FollowReferences_FollowRefObjects_addRefToVerify 00000001800016e8 f   libNonConcreteKlassFilter.obj
 0001:000008c0       Java_nsk_jvmti_unit_FollowReferences_FollowRefObjects_getTag 00000001800018c0 f   libNonConcreteKlassFilter.obj
 0001:00000980       Java_nsk_jvmti_unit_FollowReferences_FollowRefObjects_resetRefsToVerify 0000000180001980 f   libNonConcreteKlassFilter.obj
 0001:00000988       Java_nsk_jvmti_unit_FollowReferences_FollowRefObjects_resetTags 0000000180001988 f   libNonConcreteKlassFilter.obj
 0001:000009cc       Java_nsk_jvmti_unit_FollowReferences_FollowRefObjects_setTag 00000001800019cc f   libNonConcreteKlassFilter.obj
 0001:00000c24       Java_nsk_share_jvmti_ArgumentHandler_getAgentOptionsString 0000000180001c24 f   libNonConcreteKlassFilter.obj
 0001:00000cd4       Java_nsk_share_jvmti_DebugeeClass_checkStatus 0000000180001cd4 f   libNonConcreteKlassFilter.obj
 0001:00000d5c       Java_nsk_share_jvmti_DebugeeClass_resetAgentData 0000000180001d5c f   libNonConcreteKlassFilter.obj
 0001:00000dbc       Java_nsk_share_jvmti_RedefineAgent_agentStatus 0000000180001dbc f   libNonConcreteKlassFilter.obj
 0001:00000dc8       Java_nsk_share_jvmti_RedefineAgent_isRedefined 0000000180001dc8 f   libNonConcreteKlassFilter.obj
 0001:00000dd4       Java_nsk_share_jvmti_RedefineAgent_redefineAttempted 0000000180001dd4 f   libNonConcreteKlassFilter.obj
 0001:00000de0       MA_checkStatus             0000000180001de0 f   libNonConcreteKlassFilter.obj
 0001:00000e84       __local_stdio_printf_options 0000000180001e84 f i libNonConcreteKlassFilter.obj
 0001:000014b4       array_callback             00000001800024b4 f   libNonConcreteKlassFilter.obj
 0001:000016a8       exitOnError                00000001800026a8 f   libNonConcreteKlassFilter.obj
 0001:0000172c       field_callback             000000018000272c f   libNonConcreteKlassFilter.obj
 0001:00001818       fprintf                    0000000180002818 f i libNonConcreteKlassFilter.obj
 0001:0000185c       heap_callback              000000018000285c f   libNonConcreteKlassFilter.obj
 0001:0000189c       nsk_complain               000000018000289c f   libNonConcreteKlassFilter.obj
 0001:000018c8       nsk_jvmti_createJVMTIEnv   00000001800028c8 f   libNonConcreteKlassFilter.obj
 0001:000019f8       nsk_jvmti_enableEvents     00000001800029f8 f   libNonConcreteKlassFilter.obj
 0001:00001acc       nsk_jvmti_lverify          0000000180002acc f   libNonConcreteKlassFilter.obj
 0001:00001bbc       nsk_jvmti_parseOptions     0000000180002bbc f   libNonConcreteKlassFilter.obj
 0001:00001e0c       nsk_jvmti_resetAgentData   0000000180002e0c f   libNonConcreteKlassFilter.obj
 0001:00001e8c       nsk_jvmti_resumeSync       0000000180002e8c f   libNonConcreteKlassFilter.obj
 0001:00001f34       nsk_jvmti_setFailStatus    0000000180002f34 f   libNonConcreteKlassFilter.obj
 0001:00001f70       nsk_jvmti_waitForSync      0000000180002f70 f   libNonConcreteKlassFilter.obj
 0001:00002074       nsk_lcomplain              0000000180003074 f   libNonConcreteKlassFilter.obj
 0001:00002094       nsk_ldisplay               0000000180003094 f   libNonConcreteKlassFilter.obj
 0001:000020b4       nsk_ltrace                 00000001800030b4 f   libNonConcreteKlassFilter.obj
 0001:000020d4       nsk_lvcomplain             00000001800030d4 f   libNonConcreteKlassFilter.obj
 0001:0000228c       nsk_lvdisplay              000000018000328c f   libNonConcreteKlassFilter.obj
 0001:000022d8       nsk_lverify                00000001800032d8 f   libNonConcreteKlassFilter.obj
 0001:00002334       nsk_lvtrace                0000000180003334 f   libNonConcreteKlassFilter.obj
 0001:00002394       nsk_printf                 0000000180003394 f   libNonConcreteKlassFilter.obj
 0001:000023bc       nsk_vprintf                00000001800033bc f   libNonConcreteKlassFilter.obj
 0001:00002470       printf                     0000000180003470 f i libNonConcreteKlassFilter.obj
 0001:00002800       string_callback            0000000180003800 f   libNonConcreteKlassFilter.obj
 0001:000029c8       __raise_securityfailure    00000001800039c8 f   MSVCRT:gs_report.obj
 0001:000029fc       __report_gsfailure         00000001800039fc f   MSVCRT:gs_report.obj
 0001:00002c3c       __GSHandlerCheck           0000000180003c3c f   MSVCRT:gshandler.obj
 0001:00002c5c       __GSHandlerCheckCommon     0000000180003c5c f   MSVCRT:gshandler.obj
 0001:00002cd0       __security_check_cookie    0000000180003cd0 f   MSVCRT:amdsecgs.obj
 0001:00003010       _DllMainCRTStartup         0000000180004010 f   MSVCRT:dll_dllmain.obj
 0001:00003050       __scrt_acquire_startup_lock 0000000180004050 f   MSVCRT:utility.obj
 0001:0000308c       __scrt_dllmain_after_initialize_c 000000018000408c f   MSVCRT:utility.obj
 0001:000030c0       __scrt_dllmain_before_initialize_c 00000001800040c0 f   MSVCRT:utility.obj
 0001:000030d8       __scrt_dllmain_crt_thread_attach 00000001800040d8 f   MSVCRT:utility.obj
 0001:00003100       __scrt_dllmain_crt_thread_detach 0000000180004100 f   MSVCRT:utility.obj
 0001:00003118       __scrt_dllmain_exception_filter 0000000180004118 f   MSVCRT:utility.obj
 0001:00003178       __scrt_dllmain_uninitialize_c 0000000180004178 f   MSVCRT:utility.obj
 0001:000031a8       __scrt_dllmain_uninitialize_critical 00000001800041a8 f   MSVCRT:utility.obj
 0001:000031bc       __scrt_initialize_crt      00000001800041bc f   MSVCRT:utility.obj
 0001:00003208       __scrt_initialize_onexit_tables 0000000180004208 f   MSVCRT:utility.obj
 0001:00003294       __scrt_is_nonwritable_in_current_image 0000000180004294 f   MSVCRT:utility.obj
 0001:0000332c       __scrt_release_startup_lock 000000018000432c f   MSVCRT:utility.obj
 0001:00003350       __scrt_uninitialize_crt    0000000180004350 f   MSVCRT:utility.obj
 0001:0000337c       _onexit                    000000018000437c f   MSVCRT:utility.obj
 0001:000033b8       atexit                     00000001800043b8 f   MSVCRT:utility.obj
 0001:000033d0       __crt_debugger_hook        00000001800043d0 f   MSVCRT:utility_desktop.obj
 0001:000033d8       __scrt_fastfail            00000001800043d8 f   MSVCRT:utility_desktop.obj
 0001:00003524       _guard_check_icall_nop     0000000180004524 f i MSVCRT:guard_support.obj
 0001:00003528       __security_init_cookie     0000000180004528 f   MSVCRT:gs_support.obj
 0001:000035d4       DllMain                    00000001800045d4 f   MSVCRT:dll_dllmain_stub.obj
 0001:000035f8       ?__scrt_initialize_type_info@@YAXXZ 00000001800045f8 f   MSVCRT:tncleanup.obj
 0001:00003608       ?__scrt_uninitialize_type_info@@YAXXZ 0000000180004608 f   MSVCRT:tncleanup.obj
 0001:00003614       __local_stdio_scanf_options 0000000180004614 f i MSVCRT:default_local_stdio_options.obj
 0001:0000361c       __scrt_initialize_default_local_stdio_options 000000018000461c f   MSVCRT:default_local_stdio_options.obj
 0001:00003638       __scrt_get_dyn_tls_init_callback 0000000180004638 f   MSVCRT:dyn_tls_init.obj
 0001:00003640       _RTC_Initialize            0000000180004640 f   MSVCRT:initsect.obj
 0001:0000367c       _RTC_Terminate             000000018000467c f   MSVCRT:initsect.obj
 0001:000036b8       __isa_available_init       00000001800046b8 f   MSVCRT:cpu_disp.obj
 0001:00003864       _get_startup_argv_mode     0000000180004864 f   MSVCRT:argv_mode.obj
 0001:0000386c       __scrt_is_ucrt_dll_in_use  000000018000486c f   MSVCRT:ucrt_detection.obj
 0001:00003880       memcpy                     0000000180004880 f   vcruntime:VCRUNTIME140.dll
 0001:00003886       memset                     0000000180004886 f   vcruntime:VCRUNTIME140.dll
 0001:0000388c       strchr                     000000018000488c f   vcruntime:VCRUNTIME140.dll
 0001:00003892       __C_specific_handler       0000000180004892 f   vcruntime:VCRUNTIME140.dll
 0001:00003898       __std_type_info_destroy_list 0000000180004898 f   vcruntime:VCRUNTIME140.dll
 0001:0000389e       strcmp                     000000018000489e f   ucrt:api-ms-win-crt-string-l1-1-0.dll
 0001:000038a4       strlen                     00000001800048a4 f   ucrt:api-ms-win-crt-string-l1-1-0.dll
 0001:000038aa       _initterm                  00000001800048aa f   ucrt:api-ms-win-crt-runtime-l1-1-0.dll
 0001:000038b0       _initterm_e                00000001800048b0 f   ucrt:api-ms-win-crt-runtime-l1-1-0.dll
 0001:000038b6       _seh_filter_dll            00000001800048b6 f   ucrt:api-ms-win-crt-runtime-l1-1-0.dll
 0001:000038bc       _configure_narrow_argv     00000001800048bc f   ucrt:api-ms-win-crt-runtime-l1-1-0.dll
 0001:000038c2       _initialize_narrow_environment 00000001800048c2 f   ucrt:api-ms-win-crt-runtime-l1-1-0.dll
 0001:000038c8       _initialize_onexit_table   00000001800048c8 f   ucrt:api-ms-win-crt-runtime-l1-1-0.dll
 0001:000038ce       _register_onexit_function  00000001800048ce f   ucrt:api-ms-win-crt-runtime-l1-1-0.dll
 0001:000038d4       _execute_onexit_table      00000001800048d4 f   ucrt:api-ms-win-crt-runtime-l1-1-0.dll
 0001:000038da       _crt_atexit                00000001800048da f   ucrt:api-ms-win-crt-runtime-l1-1-0.dll
 0001:000038e0       _cexit                     00000001800048e0 f   ucrt:api-ms-win-crt-runtime-l1-1-0.dll
 0001:000038e8       __acrt_initialize          00000001800048e8 f   MSVCRT:ucrt_stubs.obj
 0001:000038e8       __acrt_thread_attach       00000001800048e8 f   MSVCRT:ucrt_stubs.obj
 0001:000038e8       __acrt_thread_detach       00000001800048e8 f   MSVCRT:ucrt_stubs.obj
 0001:000038e8       __acrt_uninitialize        00000001800048e8 f   MSVCRT:ucrt_stubs.obj
 0001:000038e8       __acrt_uninitialize_critical 00000001800048e8 f   MSVCRT:ucrt_stubs.obj
 0001:000038e8       __scrt_stub_for_acrt_initialize 00000001800048e8 f   MSVCRT:ucrt_stubs.obj
 0001:000038e8       __scrt_stub_for_acrt_thread_attach 00000001800048e8 f   MSVCRT:ucrt_stubs.obj
 0001:000038e8       __scrt_stub_for_acrt_thread_detach 00000001800048e8 f   MSVCRT:ucrt_stubs.obj
 0001:000038e8       __scrt_stub_for_acrt_uninitialize 00000001800048e8 f   MSVCRT:ucrt_stubs.obj
 0001:000038e8       __scrt_stub_for_acrt_uninitialize_critical 00000001800048e8 f   MSVCRT:ucrt_stubs.obj
 0001:000038e8       __vcrt_initialize          00000001800048e8 f   MSVCRT:ucrt_stubs.obj
 0001:000038e8       __vcrt_thread_attach       00000001800048e8 f   MSVCRT:ucrt_stubs.obj
 0001:000038e8       __vcrt_thread_detach       00000001800048e8 f   MSVCRT:ucrt_stubs.obj
 0001:000038e8       __vcrt_uninitialize        00000001800048e8 f   MSVCRT:ucrt_stubs.obj
 0001:000038e8       __vcrt_uninitialize_critical 00000001800048e8 f   MSVCRT:ucrt_stubs.obj
 0001:000038ec       __scrt_stub_for_is_c_termination_complete 00000001800048ec f   MSVCRT:ucrt_stubs.obj
 0001:000038ec       _is_c_termination_complete 00000001800048ec f   MSVCRT:ucrt_stubs.obj
 0001:00003900       _guard_dispatch_icall_nop  0000000180004900 f   MSVCRT:guard_dispatch.obj
 0001:00003920       _guard_xfg_dispatch_icall_nop 0000000180004920 f   MSVCRT:guard_xfg_dispatch.obj
 0002:00000000       __imp_RtlCaptureContext    0000000180005000     kernel32:KERNEL32.dll
 0002:00000008       __imp_RtlLookupFunctionEntry 0000000180005008     kernel32:KERNEL32.dll
 0002:00000010       __imp_RtlVirtualUnwind     0000000180005010     kernel32:KERNEL32.dll
 0002:00000018       __imp_UnhandledExceptionFilter 0000000180005018     kernel32:KERNEL32.dll
 0002:00000020       __imp_SetUnhandledExceptionFilter 0000000180005020     kernel32:KERNEL32.dll
 0002:00000028       __imp_GetCurrentProcess    0000000180005028     kernel32:KERNEL32.dll
 0002:00000030       __imp_TerminateProcess     0000000180005030     kernel32:KERNEL32.dll
 0002:00000038       __imp_IsProcessorFeaturePresent 0000000180005038     kernel32:KERNEL32.dll
 0002:00000040       __imp_CloseHandle          0000000180005040     kernel32:KERNEL32.dll
 0002:00000048       __imp_InitializeCriticalSectionAndSpinCount 0000000180005048     kernel32:KERNEL32.dll
 0002:00000050       __imp_DeleteCriticalSection 0000000180005050     kernel32:KERNEL32.dll
 0002:00000058       __imp_CreateEventW         0000000180005058     kernel32:KERNEL32.dll
 0002:00000060       __imp_GetModuleHandleW     0000000180005060     kernel32:KERNEL32.dll
 0002:00000068       __imp_GetProcAddress       0000000180005068     kernel32:KERNEL32.dll
 0002:00000070       __imp_IsDebuggerPresent    0000000180005070     kernel32:KERNEL32.dll
 0002:00000078       __imp_QueryPerformanceCounter 0000000180005078     kernel32:KERNEL32.dll
 0002:00000080       __imp_GetCurrentProcessId  0000000180005080     kernel32:KERNEL32.dll
 0002:00000088       __imp_GetCurrentThreadId   0000000180005088     kernel32:KERNEL32.dll
 0002:00000090       __imp_GetSystemTimeAsFileTime 0000000180005090     kernel32:KERNEL32.dll
 0002:00000098       __imp_DisableThreadLibraryCalls 0000000180005098     kernel32:KERNEL32.dll
 0002:000000a0       __imp_InitializeSListHead  00000001800050a0     kernel32:KERNEL32.dll
 0002:000000a8       \177KERNEL32_NULL_THUNK_DATA 00000001800050a8     kernel32:KERNEL32.dll
 0002:000000b0       __imp_memcpy               00000001800050b0     vcruntime:VCRUNTIME140.dll
 0002:000000b8       __imp_memset               00000001800050b8     vcruntime:VCRUNTIME140.dll
 0002:000000c0       __imp_strchr               00000001800050c0     vcruntime:VCRUNTIME140.dll
 0002:000000c8       __imp___C_specific_handler 00000001800050c8     vcruntime:VCRUNTIME140.dll
 0002:000000d0       __imp___std_type_info_destroy_list 00000001800050d0     vcruntime:VCRUNTIME140.dll
 0002:000000d8       \177VCRUNTIME140_NULL_THUNK_DATA 00000001800050d8     vcruntime:VCRUNTIME140.dll
 0002:000000e0       __imp_strtol               00000001800050e0     ucrt:api-ms-win-crt-convert-l1-1-0.dll
 0002:000000e8       \177api-ms-win-crt-convert-l1-1-0_NULL_THUNK_DATA 00000001800050e8     ucrt:api-ms-win-crt-convert-l1-1-0.dll
 0002:000000f0       __imp_malloc               00000001800050f0     ucrt:api-ms-win-crt-heap-l1-1-0.dll
 0002:000000f8       __imp_free                 00000001800050f8     ucrt:api-ms-win-crt-heap-l1-1-0.dll
 0002:00000100       \177api-ms-win-crt-heap-l1-1-0_NULL_THUNK_DATA 0000000180005100     ucrt:api-ms-win-crt-heap-l1-1-0.dll
 0002:00000108       __imp__errno               0000000180005108     ucrt:api-ms-win-crt-runtime-l1-1-0.dll
 0002:00000110       __imp_exit                 0000000180005110     ucrt:api-ms-win-crt-runtime-l1-1-0.dll
 0002:00000118       __imp__cexit               0000000180005118     ucrt:api-ms-win-crt-runtime-l1-1-0.dll
 0002:00000120       __imp__crt_atexit          0000000180005120     ucrt:api-ms-win-crt-runtime-l1-1-0.dll
 0002:00000128       __imp__execute_onexit_table 0000000180005128     ucrt:api-ms-win-crt-runtime-l1-1-0.dll
 0002:00000130       __imp__register_onexit_function 0000000180005130     ucrt:api-ms-win-crt-runtime-l1-1-0.dll
 0002:00000138       __imp__initialize_onexit_table 0000000180005138     ucrt:api-ms-win-crt-runtime-l1-1-0.dll
 0002:00000140       __imp__initialize_narrow_environment 0000000180005140     ucrt:api-ms-win-crt-runtime-l1-1-0.dll
 0002:00000148       __imp__configure_narrow_argv 0000000180005148     ucrt:api-ms-win-crt-runtime-l1-1-0.dll
 0002:00000150       __imp__seh_filter_dll      0000000180005150     ucrt:api-ms-win-crt-runtime-l1-1-0.dll
 0002:00000158       __imp__initterm_e          0000000180005158     ucrt:api-ms-win-crt-runtime-l1-1-0.dll
 0002:00000160       __imp__initterm            0000000180005160     ucrt:api-ms-win-crt-runtime-l1-1-0.dll
 0002:00000168       \177api-ms-win-crt-runtime-l1-1-0_NULL_THUNK_DATA 0000000180005168     ucrt:api-ms-win-crt-runtime-l1-1-0.dll
 0002:00000170       __imp___acrt_iob_func      0000000180005170     ucrt:api-ms-win-crt-stdio-l1-1-0.dll
 0002:00000178       __imp_fflush               0000000180005178     ucrt:api-ms-win-crt-stdio-l1-1-0.dll
 0002:00000180       __imp___stdio_common_vsprintf 0000000180005180     ucrt:api-ms-win-crt-stdio-l1-1-0.dll
 0002:00000188       __imp___stdio_common_vfprintf 0000000180005188     ucrt:api-ms-win-crt-stdio-l1-1-0.dll
 0002:00000190       \177api-ms-win-crt-stdio-l1-1-0_NULL_THUNK_DATA 0000000180005190     ucrt:api-ms-win-crt-stdio-l1-1-0.dll
 0002:00000198       __imp_strcmp               0000000180005198     ucrt:api-ms-win-crt-string-l1-1-0.dll
 0002:000001a0       __imp__strdup              00000001800051a0     ucrt:api-ms-win-crt-string-l1-1-0.dll
 0002:000001a0       __imp_strdup               00000001800051a0     ucrt:api-ms-win-crt-string-l1-1-0.dll
 0002:000001a8       __imp_strlen               00000001800051a8     ucrt:api-ms-win-crt-string-l1-1-0.dll
 0002:000001b0       __imp_strpbrk              00000001800051b0     ucrt:api-ms-win-crt-string-l1-1-0.dll
 0002:000001b8       __imp_strncpy              00000001800051b8     ucrt:api-ms-win-crt-string-l1-1-0.dll
 0002:000001c0       \177api-ms-win-crt-string-l1-1-0_NULL_THUNK_DATA 00000001800051c0     ucrt:api-ms-win-crt-string-l1-1-0.dll
 0002:000001c8       __guard_check_icall_fptr   00000001800051c8     MSVCRT:guard_support.obj
 0002:000001d0       __guard_xfg_check_icall_fptr 00000001800051d0     MSVCRT:guard_support.obj
 0002:000001d8       __guard_dispatch_icall_fptr 00000001800051d8     MSVCRT:guard_support.obj
 0002:000001e0       __guard_xfg_dispatch_icall_fptr 00000001800051e0     MSVCRT:guard_support.obj
 0002:000001e8       __guard_xfg_table_dispatch_icall_fptr 00000001800051e8     MSVCRT:guard_support.obj
 0002:000001f0       __castguard_check_failure_os_handled_fptr 00000001800051f0     MSVCRT:guard_support.obj
 0002:000001f8       __guard_memcpy_fptr        00000001800051f8     vcruntime:softmemtag.obj
 0002:00000200       __xc_a                     0000000180005200     MSVCRT:initializers.obj
 0002:00000208       __xc_z                     0000000180005208     MSVCRT:initializers.obj
 0002:00000210       __xi_a                     0000000180005210     MSVCRT:initializers.obj
 0002:00000220       __xi_z                     0000000180005220     MSVCRT:initializers.obj
 0002:00000228       __xl_a                     0000000180005228     MSVCRT:tlssup.obj
 0002:00000230       __xl_z                     0000000180005230     MSVCRT:tlssup.obj
 0002:00000238       __xp_a                     0000000180005238     MSVCRT:initializers.obj
 0002:00000240       __xp_z                     0000000180005240     MSVCRT:initializers.obj
 0002:00000248       __xt_a                     0000000180005248     MSVCRT:initializers.obj
 0002:00000250       __xt_z                     0000000180005250     MSVCRT:initializers.obj
 0002:00000260       g_refKindStr               0000000180005260     libNonConcreteKlassFilter.obj
 0002:00000410       ??_C@_09BPLDFGCI@unknown_0@ 0000000180005410     libNonConcreteKlassFilter.obj
 0002:00000420       ??_C@_0BL@FPNMECJD@JVMTI_HEAP_REFERENCE_CLASS@ 0000000180005420     libNonConcreteKlassFilter.obj
 0002:00000440       ??_C@_0BL@FKGKKLNM@JVMTI_HEAP_REFERENCE_FIELD@ 0000000180005440     libNonConcreteKlassFilter.obj
 0002:00000460       ??_C@_0CD@CAEHCFJF@JVMTI_HEAP_REFERENCE_ARRAY_ELEM@ 0000000180005460     libNonConcreteKlassFilter.obj
 0002:00000488       ??_C@_0CC@DNEBMCNK@JVMTI_HEAP_REFERENCE_CLASS_LOAD@ 0000000180005488     libNonConcreteKlassFilter.obj
 0002:000004b0       ??_C@_0BN@CJMIPEBB@JVMTI_HEAP_REFERENCE_SIGNERS@ 00000001800054b0     libNonConcreteKlassFilter.obj
 0002:000004d0       ??_C@_0CH@HBOIDPEB@JVMTI_HEAP_REFERENCE_PROTECTION@ 00000001800054d0     libNonConcreteKlassFilter.obj
 0002:000004f8       ??_C@_0BP@MDKGDGKL@JVMTI_HEAP_REFERENCE_INTERFACE@ 00000001800054f8     libNonConcreteKlassFilter.obj
 0002:00000518       ??_C@_0CC@JJMIHNJH@JVMTI_HEAP_REFERENCE_STATIC_FIE@ 0000000180005518     libNonConcreteKlassFilter.obj
 0002:00000540       ??_C@_0CD@IDHEEGID@JVMTI_HEAP_REFERENCE_CONSTANT_P@ 0000000180005540     libNonConcreteKlassFilter.obj
 0002:00000568       ??_C@_0CA@EFFCHNG@JVMTI_HEAP_REFERENCE_SUPERCLASS@ 0000000180005568     libNonConcreteKlassFilter.obj
 0002:00000588       ??_C@_0L@PCDFHGCJ@unknown_11@ 0000000180005588     libNonConcreteKlassFilter.obj
 0002:00000598       ??_C@_0L@NJBICFOK@unknown_12@ 0000000180005598     libNonConcreteKlassFilter.obj
 0002:000005a8       ??_C@_0L@MAADBEKL@unknown_13@ 00000001800055a8     libNonConcreteKlassFilter.obj
 0002:000005b8       ??_C@_0L@IPECICGM@unknown_14@ 00000001800055b8     libNonConcreteKlassFilter.obj
 0002:000005c8       ??_C@_0L@JGFJLDCN@unknown_15@ 00000001800055c8     libNonConcreteKlassFilter.obj
 0002:000005d8       ??_C@_0L@LNHEOAOO@unknown_16@ 00000001800055d8     libNonConcreteKlassFilter.obj
 0002:000005e8       ??_C@_0L@KEGPNBKP@unknown_17@ 00000001800055e8     libNonConcreteKlassFilter.obj
 0002:000005f8       ??_C@_0L@CDPHMNGA@unknown_18@ 00000001800055f8     libNonConcreteKlassFilter.obj
 0002:00000608       ??_C@_0L@DKOMPMCB@unknown_19@ 0000000180005608     libNonConcreteKlassFilter.obj
 0002:00000618       ??_C@_0L@OJGIPJDB@unknown_20@ 0000000180005618     libNonConcreteKlassFilter.obj
 0002:00000628       ??_C@_0CA@KAOFNDEM@JVMTI_HEAP_REFERENCE_JNI_GLOBAL@ 0000000180005628     libNonConcreteKlassFilter.obj
 0002:00000648       ??_C@_0CC@HPFAJBK@JVMTI_HEAP_REFERENCE_SYSTEM_CLA@ 0000000180005648     libNonConcreteKlassFilter.obj
 0002:00000670       ??_C@_0BN@FDEGFOHC@JVMTI_HEAP_REFERENCE_MONITOR@ 0000000180005670     libNonConcreteKlassFilter.obj
 0002:00000690       ??_C@_0CB@HKIBCMAJ@JVMTI_HEAP_REFERENCE_STACK_LOCA@ 0000000180005690     libNonConcreteKlassFilter.obj
 0002:000006b8       ??_C@_0BP@EAACMMOE@JVMTI_HEAP_REFERENCE_JNI_LOCAL@ 00000001800056b8     libNonConcreteKlassFilter.obj
 0002:000006d8       ??_C@_0BM@IJDEOGOE@JVMTI_HEAP_REFERENCE_THREAD@ 00000001800056d8     libNonConcreteKlassFilter.obj
 0002:000006f8       ??_C@_0BL@EDGPPKC@JVMTI_HEAP_REFERENCE_OTHER@ 00000001800056f8     libNonConcreteKlassFilter.obj
 0002:00000714       ??_C@_04BCJPDBDA@Code@     0000000180005714     libNonConcreteKlassFilter.obj
 0002:00000720       ??_C@_0BA@OCLMCFKC@LineNumberTable@ 0000000180005720     libNonConcreteKlassFilter.obj
 0002:00000730       ??_C@_0BD@CPAEPILC@LocalVariableTable@ 0000000180005730     libNonConcreteKlassFilter.obj
 0002:00000748       ??_C@_0BH@NMBDNHBD@LocalVariableTypeTable@ 0000000180005748     libNonConcreteKlassFilter.obj
 0002:00000760       ??_C@_0O@HIHEEDNJ@StackMapTable@ 0000000180005760     libNonConcreteKlassFilter.obj
 0002:00000770       ??_C@_0EB@PMMMPCEL@nsk?1jvmti?1IterateThroughHeap?1no@ 0000000180005770     libNonConcreteKlassFilter.obj
 0002:000007c0       ??_C@_0EF@EDCHNDHH@nsk?1jvmti?1IterateThroughHeap?1no@ 00000001800057c0     libNonConcreteKlassFilter.obj
 0002:00000808       ??_C@_0L@HCDIAMJG@?9?5?$CFs?0?5?$CFd?3?5@ 0000000180005808     libNonConcreteKlassFilter.obj
 0002:00000820       ??_C@_0JI@HLPECLFI@?$CD?5?4?4?4?6?$CD?5ERROR?3?5too?5many?5complai@ 0000000180005820     libNonConcreteKlassFilter.obj
 0002:000008c0       ??_C@_0ED@JNEKCCOB@The?5following?5fake?5exception?5st@ 00000001800058c0     libNonConcreteKlassFilter.obj
 0002:00000908       ??_C@_0CN@FCNMDFBH@nsk?4share?4Fake_Exception_for_RU@ 0000000180005908     libNonConcreteKlassFilter.obj
 0002:00000938       ??_C@_08PGFFNAEI@?$CI?$CFs?3?$CFd?$CJ?5@ 0000000180005938     libNonConcreteKlassFilter.obj
 0002:00000948       ??_C@_0DP@IENMAEGI@s?2test?2hotspot?2jtreg?2vmTestbase@ 0000000180005948     libNonConcreteKlassFilter.obj
 0002:00000988       ??_C@_0BL@NDJLFFJB@?7at?5nsk_lvcomplain?$CI?$CFs?3?$CFd?$CJ?6@ 0000000180005988     libNonConcreteKlassFilter.obj
 0002:000009a8       ??_C@_0BC@JOOKAFKF@?$CD?5ERROR?3?5?$CFs?0?5?$CFd?3?5@ 00000001800059a8     libNonConcreteKlassFilter.obj
 0002:000009c0       ??_C@_09KJEAHMEH@?$CD?5ERROR?3?5@ 00000001800059c0     libNonConcreteKlassFilter.obj
 0002:000009cc       ??_C@_02GPIOPFAK@?$DO?$DO@ 00000001800059cc     libNonConcreteKlassFilter.obj
 0002:000009d0       ??_C@_02FODMEDOG@?$DM?$DM@ 00000001800059d0     libNonConcreteKlassFilter.obj
 0002:000009d4       ??_C@_02DJGKEECL@?4?4@     00000001800059d4     libNonConcreteKlassFilter.obj
 0002:000009d8       ??_C@_0O@CJPGJOAF@?9?5?$CFs?0?5?$CFd?3?5?$CFs?5@ 00000001800059d8     libNonConcreteKlassFilter.obj
 0002:000009e8       ??_C@_0CB@IAKPDOIC@?$CD?5?5?5verified?5assertion?5is?5FALSE@ 00000001800059e8     libNonConcreteKlassFilter.obj
 0002:00000a10       ??_C@_0CO@LGONDEPD@stdout?3?5fflush?5failed?5?9?5err?$DN?$CFd?5@ 0000000180005a10     libNonConcreteKlassFilter.obj
 0002:00000a40       ??_C@_0CO@KBGKJPBD@stderr?3?5fflush?5failed?5?9?5err?$DN?$CFd?5@ 0000000180005a40     libNonConcreteKlassFilter.obj
 0002:00000a70       ??_C@_0BB@JCNMKLLK@JVMTI_ERROR_NONE@ 0000000180005a70     libNonConcreteKlassFilter.obj
 0002:00000a88       ??_C@_0BL@LDIMKLPH@JVMTI_ERROR_INVALID_THREAD@ 0000000180005a88     libNonConcreteKlassFilter.obj
 0002:00000aa8       ??_C@_0CB@PJFPAIKJ@JVMTI_ERROR_INVALID_THREAD_GROU@ 0000000180005aa8     libNonConcreteKlassFilter.obj
 0002:00000ad0       ??_C@_0BN@LLMKHMNF@JVMTI_ERROR_INVALID_PRIORITY@ 0000000180005ad0     libNonConcreteKlassFilter.obj
 0002:00000af0       ??_C@_0CB@MBOFKAGB@JVMTI_ERROR_THREAD_NOT_SUSPENDE@ 0000000180005af0     libNonConcreteKlassFilter.obj
 0002:00000b18       ??_C@_0BN@FABOLPBI@JVMTI_ERROR_THREAD_SUSPENDED@ 0000000180005b18     libNonConcreteKlassFilter.obj
 0002:00000b38       ??_C@_0BN@FDGNOBJM@JVMTI_ERROR_THREAD_NOT_ALIVE@ 0000000180005b38     libNonConcreteKlassFilter.obj
 0002:00000b58       ??_C@_0BL@GOBIFKNJ@JVMTI_ERROR_INVALID_OBJECT@ 0000000180005b58     libNonConcreteKlassFilter.obj
 0002:00000b78       ??_C@_0BK@FCMAJPPC@JVMTI_ERROR_INVALID_CLASS@ 0000000180005b78     libNonConcreteKlassFilter.obj
 0002:00000b98       ??_C@_0BP@IKLLBKEB@JVMTI_ERROR_CLASS_NOT_PREPARED@ 0000000180005b98     libNonConcreteKlassFilter.obj
 0002:00000bb8       ??_C@_0BN@KLPPLKG@JVMTI_ERROR_INVALID_METHODID@ 0000000180005bb8     libNonConcreteKlassFilter.obj
 0002:00000bd8       ??_C@_0BN@BCEKOKND@JVMTI_ERROR_INVALID_LOCATION@ 0000000180005bd8     libNonConcreteKlassFilter.obj
 0002:00000bf8       ??_C@_0BM@DFDGPME@JVMTI_ERROR_INVALID_FIELDID@ 0000000180005bf8     libNonConcreteKlassFilter.obj
 0002:00000c18       ??_C@_0BL@NELIEPEC@JVMTI_ERROR_NO_MORE_FRAMES@ 0000000180005c18     libNonConcreteKlassFilter.obj
 0002:00000c38       ??_C@_0BJ@BDBECFDM@JVMTI_ERROR_OPAQUE_FRAME@ 0000000180005c38     libNonConcreteKlassFilter.obj
 0002:00000c58       ??_C@_0BK@MIIFNLOB@JVMTI_ERROR_TYPE_MISMATCH@ 0000000180005c58     libNonConcreteKlassFilter.obj
 0002:00000c78       ??_C@_0BJ@HPCAOILC@JVMTI_ERROR_INVALID_SLOT@ 0000000180005c78     libNonConcreteKlassFilter.obj
 0002:00000c98       ??_C@_0BG@CHILOPNI@JVMTI_ERROR_DUPLICATE@ 0000000180005c98     libNonConcreteKlassFilter.obj
 0002:00000cb0       ??_C@_0BG@DIEMLHKM@JVMTI_ERROR_NOT_FOUND@ 0000000180005cb0     libNonConcreteKlassFilter.obj
 0002:00000cc8       ??_C@_0BM@NHMCKHOB@JVMTI_ERROR_INVALID_MONITOR@ 0000000180005cc8     libNonConcreteKlassFilter.obj
 0002:00000ce8       ??_C@_0BO@PPEDAJGL@JVMTI_ERROR_NOT_MONITOR_OWNER@ 0000000180005ce8     libNonConcreteKlassFilter.obj
 0002:00000d08       ??_C@_0BG@FCAIPEID@JVMTI_ERROR_INTERRUPT@ 0000000180005d08     libNonConcreteKlassFilter.obj
 0002:00000d20       ??_C@_0CB@EGDBNKOI@JVMTI_ERROR_INVALID_CLASS_FORMA@ 0000000180005d20     libNonConcreteKlassFilter.obj
 0002:00000d48       ??_C@_0CG@DGKOGIAL@JVMTI_ERROR_CIRCULAR_CLASS_DEFI@ 0000000180005d48     libNonConcreteKlassFilter.obj
 0002:00000d70       ??_C@_0BP@ICEALPKC@JVMTI_ERROR_FAILS_VERIFICATION@ 0000000180005d70     libNonConcreteKlassFilter.obj
 0002:00000d90       ??_C@_0DC@JDACLMIO@JVMTI_ERROR_UNSUPPORTED_REDEFIN@ 0000000180005d90     libNonConcreteKlassFilter.obj
 0002:00000dc8       ??_C@_0DE@GKDKNOMJ@JVMTI_ERROR_UNSUPPORTED_REDEFIN@ 0000000180005dc8     libNonConcreteKlassFilter.obj
 0002:00000e00       ??_C@_0BO@LAFKIOG@JVMTI_ERROR_INVALID_TYPESTATE@ 0000000180005e00     libNonConcreteKlassFilter.obj
 0002:00000e20       ??_C@_0DH@INDGCLLB@JVMTI_ERROR_UNSUPPORTED_REDEFIN@ 0000000180005e20     libNonConcreteKlassFilter.obj
 0002:00000e58       ??_C@_0DE@NHEOMMGI@JVMTI_ERROR_UNSUPPORTED_REDEFIN@ 0000000180005e58     libNonConcreteKlassFilter.obj
 0002:00000e90       ??_C@_0CA@EKPNJOEP@JVMTI_ERROR_UNSUPPORTED_VERSION@ 0000000180005e90     libNonConcreteKlassFilter.obj
 0002:00000eb0       ??_C@_0BN@OFFMAHHL@JVMTI_ERROR_NAMES_DONT_MATCH@ 0000000180005eb0     libNonConcreteKlassFilter.obj
 0002:00000ed0       ??_C@_0DN@HHBBLAKE@JVMTI_ERROR_UNSUPPORTED_REDEFIN@ 0000000180005ed0     libNonConcreteKlassFilter.obj
 0002:00000f10       ??_C@_0DO@HMBGBGNA@JVMTI_ERROR_UNSUPPORTED_REDEFIN@ 0000000180005f10     libNonConcreteKlassFilter.obj
 0002:00000f50       ??_C@_0BP@PBECGKHJ@JVMTI_ERROR_UNMODIFIABLE_CLASS@ 0000000180005f50     libNonConcreteKlassFilter.obj
 0002:00000f70       ??_C@_0BK@CANILEHF@JVMTI_ERROR_NOT_AVAILABLE@ 0000000180005f70     libNonConcreteKlassFilter.obj
 0002:00000f90       ??_C@_0CE@INJKMEFK@JVMTI_ERROR_MUST_POSSESS_CAPABI@ 0000000180005f90     libNonConcreteKlassFilter.obj
 0002:00000fb8       ??_C@_0BJ@LBFPFPDM@JVMTI_ERROR_NULL_POINTER@ 0000000180005fb8     libNonConcreteKlassFilter.obj
 0002:00000fd8       ??_C@_0BP@CHJPNNEM@JVMTI_ERROR_ABSENT_INFORMATION@ 0000000180005fd8     libNonConcreteKlassFilter.obj
 0002:00000ff8       ??_C@_0BP@OMFMNLC@JVMTI_ERROR_INVALID_EVENT_TYPE@ 0000000180005ff8     libNonConcreteKlassFilter.obj
 0002:00001018       ??_C@_0BN@BIBNPHHO@JVMTI_ERROR_ILLEGAL_ARGUMENT@ 0000000180006018     libNonConcreteKlassFilter.obj
 0002:00001038       ??_C@_0BK@KKNDHDCE@JVMTI_ERROR_NATIVE_METHOD@ 0000000180006038     libNonConcreteKlassFilter.obj
 0002:00001058       ??_C@_0BK@PMKCFHAE@JVMTI_ERROR_OUT_OF_MEMORY@ 0000000180006058     libNonConcreteKlassFilter.obj
 0002:00001078       ??_C@_0BK@NNJBDMNB@JVMTI_ERROR_ACCESS_DENIED@ 0000000180006078     libNonConcreteKlassFilter.obj
 0002:00001098       ??_C@_0BI@GHECLMNC@JVMTI_ERROR_WRONG_PHASE@ 0000000180006098     libNonConcreteKlassFilter.obj
 0002:000010b0       ??_C@_0BF@OLIHJOII@JVMTI_ERROR_INTERNAL@ 00000001800060b0     libNonConcreteKlassFilter.obj
 0002:000010c8       ??_C@_0BO@EOHGKJHI@JVMTI_ERROR_UNATTACHED_THREAD@ 00000001800060c8     libNonConcreteKlassFilter.obj
 0002:000010e8       ??_C@_0CA@LKHFDACL@JVMTI_ERROR_INVALID_ENVIRONMENT@ 00000001800060e8     libNonConcreteKlassFilter.obj
 0002:00001108       ??_C@_0BA@MMFHLOKK@?$DMunknown?5error?$DO@ 0000000180006108     libNonConcreteKlassFilter.obj
 0002:00001118       ??_C@_0CF@CBHOKDB@throwable?5?$DN?5jni?9?$DOExceptionOccur@ 0000000180006118     libNonConcreteKlassFilter.obj
 0002:00001140       ??_C@_03OFAPEBGM@?$CFs?6@  0000000180006140     libNonConcreteKlassFilter.obj
 0002:00001148       ??_C@_0DM@LPIGEGNJ@s?2test?2hotspot?2jtreg?2vmTestbase@ 0000000180006148     libNonConcreteKlassFilter.obj
 0002:00001188       ??_C@_0CC@NFCNPEPK@Exception?5in?5JNI?5call?5?$CIcleared?$CJ@ 0000000180006188     libNonConcreteKlassFilter.obj
 0002:000011b0       ??_C@_0BJ@IBAKFIKF@jni?9?$DOExceptionDescribe?$CI?$CJ@ 00000001800061b0     libNonConcreteKlassFilter.obj
 0002:000011d0       ??_C@_0BG@GGKALKMH@jni?9?$DOExceptionClear?$CI?$CJ@ 00000001800061d0     libNonConcreteKlassFilter.obj
 0002:000011e8       ??_C@_0CF@JMGFGJLJ@?$CD?5?5?5verified?5JNI?5assertion?5is?5F@ 00000001800061e8     libNonConcreteKlassFilter.obj
 0002:00001210       ??_C@_07KBAMPNJK@verbose@  0000000180006210     libNonConcreteKlassFilter.obj
 0002:00001218       ??_C@_0DN@PKJBOLAP@nsk_jvmti_parseOptions?$CI?$CJ?3?5unexp@ 0000000180006218     libNonConcreteKlassFilter.obj
 0002:00001258       ??_C@_05IMBNNINJ@trace@    0000000180006258     libNonConcreteKlassFilter.obj
 0002:00001260       ??_C@_0DD@BJKGNDMB@nsk_jvmti_parseOptions?$CI?$CJ?3?5no?5va@ 0000000180006260     libNonConcreteKlassFilter.obj
 0002:00001294       ??_C@_04CGFJFPFD@none@     0000000180006294     libNonConcreteKlassFilter.obj
 0002:0000129c       ??_C@_06BMELKFMA@before@   000000018000629c     libNonConcreteKlassFilter.obj
 0002:000012a4       ??_C@_05CMKPCFDK@after@    00000001800062a4     libNonConcreteKlassFilter.obj
 0002:000012ac       ??_C@_03NFKEKGGK@all@      00000001800062ac     libNonConcreteKlassFilter.obj
 0002:000012b0       ??_C@_0DM@NDNJGJKE@nsk_jvmti_parseOptions?$CI?$CJ?3?5uexpe@ 00000001800062b0     libNonConcreteKlassFilter.obj
 0002:000012f0       ??_C@_08NBBJKJO@waittime@  00000001800062f0     libNonConcreteKlassFilter.obj
 0002:00001300       ??_C@_0DO@CMHGAOHC@nsk_jvmti_parseOptions?$CI?$CJ?3?5not?5i@ 0000000180006300     libNonConcreteKlassFilter.obj
 0002:00001340       ??_C@_0DL@LNMPBDLN@nsk_jvmti_parseOptions?$CI?$CJ?3?5negat@ 0000000180006340     libNonConcreteKlassFilter.obj
 0002:00001380       ??_C@_0DA@GMFJNOJH@nsk_jvmti_parseOptions?$CI?$CJ?3?5unkno@ 0000000180006380     libNonConcreteKlassFilter.obj
 0002:000013b0       ??_C@_0CO@CCIAMEAN@nsk_jvmti_parseOptions?$CI?$CJ?3?5found@ 00000001800063b0     libNonConcreteKlassFilter.obj
 0002:000013e0       ??_C@_0CJ@OEGPCGDL@nsk_jvmti_parseOptions?$CI?$CJ?3?5out?5o@ 00000001800063e0     libNonConcreteKlassFilter.obj
 0002:00001410       ??_C@_0DI@NMBHPGGF@nsk_jvmti_parseOptions?$CI?$CJ?3?5too?5m@ 0000000180006410     libNonConcreteKlassFilter.obj
 0002:00001448       ??_C@_03POGCGECB@?5?0?$HO@ 0000000180006448     libNonConcreteKlassFilter.obj
 0002:00001450       ??_C@_0CB@MLNJNCLJ@?5?5jvmti?5error?3?5code?$DN?$CFd?0?5name?$DN?$CFs@ 0000000180006450     libNonConcreteKlassFilter.obj
 0002:00001478       ??_C@_0CD@OHBGDKMK@?$CD?5?5?5jvmti?5error?3?5code?$DN?$CFd?0?5name?$DN@ 0000000180006478     libNonConcreteKlassFilter.obj
 0002:000014a0       ??_C@_0CG@JNNCGPHB@?$CD?5?5?5error?5expected?3?5code?$DN?$CFd?0?5na@ 00000001800064a0     libNonConcreteKlassFilter.obj
 0002:000014d0       ??_C@_0EB@IMGKPCGE@?$CIstr_obj?5?$DN?5jni?9?$DONewStringUTF?$CIco@ 00000001800064d0     libNonConcreteKlassFilter.obj
 0002:00001520       ??_C@_0EA@HFOGGBCC@s?2test?2hotspot?2jtreg?2vmTestbase@ 0000000180006520     libNonConcreteKlassFilter.obj
 0002:00001560       ??_C@_05KKCIMGE@error@     0000000180006560     libNonConcreteKlassFilter.obj
 0002:00001568       ??_C@_0CJ@JACLEAA@Test?5failed?5by?5setFailStatus?$CI?$CJ?4@ 0000000180006568     libNonConcreteKlassFilter.obj
 0002:00001598       ??_C@_0BD@HGNAOMCP@agent_data_monitor@ 0000000180006598     libNonConcreteKlassFilter.obj
 0002:000015b0       ??_C@_0EB@OGCLGKLN@javaVM?9?$DOGetEnv?$CI?$CIvoid?5?$CK?$CK?$CJ?$CGjvmti_@ 00000001800065b0     libNonConcreteKlassFilter.obj
 0002:00001600       ??_C@_0EA@PNBCDMOA@s?2test?2hotspot?2jtreg?2vmTestbase@ 0000000180006600     libNonConcreteKlassFilter.obj
 0002:00001640       ??_C@_0CI@DDPIFBGM@init_agent_data?$CIjvmti_env?0?5?$CGage@ 0000000180006640     libNonConcreteKlassFilter.obj
 0002:00001668       ??_C@_0DI@ILAHDLMP@?$CI?$CKagentThreadProc?$CJ?$CIjvmti_env?0?5a@ 0000000180006668     libNonConcreteKlassFilter.obj
 0002:000016a0       ??_C@_0BD@KDBALNLB@JVMTI?5agent?5thread@ 00000001800066a0     libNonConcreteKlassFilter.obj
 0002:000016b8       ??_C@_0BB@NOKBFPFO@java?1lang?1Thread@ 00000001800066b8     libNonConcreteKlassFilter.obj
 0002:000016cc       ??_C@_06FALKBLGB@?$DMinit?$DO@ 00000001800066cc     libNonConcreteKlassFilter.obj
 0002:000016d8       ??_C@_0BG@IKDDPPGD@?$CILjava?1lang?1String?$DL?$CJV@ 00000001800066d8     libNonConcreteKlassFilter.obj
 0002:000016f0       ??_C@_0EB@IFJBFEKC@?$CIthreadClass?5?$DN?5jni_env?9?$DOFindCla@ 00000001800066f0     libNonConcreteKlassFilter.obj
 0002:00001740       ??_C@_0GF@FGFIBKKL@?$CIthreadCtor?5?$DN?5jni_env?9?$DOGetMetho@ 0000000180006740     libNonConcreteKlassFilter.obj
 0002:000017a8       ??_C@_0DN@NCPDJLOG@?$CIthreadName?5?$DN?5jni_env?9?$DONewStrin@ 00000001800067a8     libNonConcreteKlassFilter.obj
 0002:000017f0       ??_C@_0FE@PFKODBGC@?$CIthreadObject?5?$DN?5jni_env?9?$DONewObj@ 00000001800067f0     libNonConcreteKlassFilter.obj
 0002:00001850       ??_C@_0ED@HOBAHHJI@?$CIthreadGlobalRef?5?$DN?5jni_env?9?$DONew@ 0000000180006850     libNonConcreteKlassFilter.obj
 0002:000018a0       ??_C@_0FN@HNJJAHFC@jvmti_env?9?$DORunAgentThread?$CIagent@ 00000001800068a0     libNonConcreteKlassFilter.obj
 0002:00001900       ??_C@_0EA@MOJDNKDF@Debuggee?5status?5sync?5aborted?5be@ 0000000180006900     libNonConcreteKlassFilter.obj
 0002:00001940       ??_C@_0CO@PGPGMHBJ@No?5status?5sync?5occured?5for?5time@ 0000000180006940     libNonConcreteKlassFilter.obj
 0002:00001970       ??_C@_0CL@DOEBDPKJ@Debuggee?5was?5not?5suspended?5on?5s@ 0000000180006970     libNonConcreteKlassFilter.obj
 0002:000019a0       ??_C@_0EA@EEOEJAEN@status?5?$DN?5syncDebuggeeStatus?$CIjni@ 00000001800069a0     libNonConcreteKlassFilter.obj
 0002:000019e0       ??_C@_0BL@JBCFNBMB@nsk_jvmti_resetAgentData?$CI?$CJ@ 00000001800069e0     libNonConcreteKlassFilter.obj
 0002:00001a00       ??_C@_0DN@NNGECJON@jvmti_env?9?$DOSetEventNotification@ 0000000180006a00     libNonConcreteKlassFilter.obj
 0002:00001a40       ??_C@_0EL@LPBEELIP@s?2test?2hotspot?2jtreg?2vmTestbase@ 0000000180006a40     libNonConcreteKlassFilter.obj
 0002:00001a90       ??_C@_0CK@JDAMFDMJ@jvmti?9?$DOSetTag?$CIo?0?5tag?$CJ?5?$DN?$DN?5JVMTI_@ 0000000180006a90     libNonConcreteKlassFilter.obj
 0002:00001ac0       ??_C@_0CC@DAMNHKNI@Can?8t?5set?5tag?5?$CFli?5for?5object?5?$CFl@ 0000000180006ac0     libNonConcreteKlassFilter.obj
 0002:00001ae8       ??_C@_0DL@HAJPNKEF@jvmti?9?$DOGetObjectHashCode?$CIo?0?5?$CGha@ 0000000180006ae8     libNonConcreteKlassFilter.obj
 0002:00001b28       ??_C@_0BL@JFPIEOBF@Can?8t?5get?5hash?5object?5?$CFlx?6@ 0000000180006b28     libNonConcreteKlassFilter.obj
 0002:00001b48       ??_C@_0BG@DICPHBKN@setTag?3?5?$CF08x?5?$DM?9?5?$CF?53li@ 0000000180006b48     libNonConcreteKlassFilter.obj
 0002:00001b60       ??_C@_0DH@FCEEBDMJ@?$CIs?5?$DN?5jni?9?$DOGetStringUTFChars?$CIsIn@ 0000000180006b60     libNonConcreteKlassFilter.obj
 0002:00001b98       ??_C@_0BJ@OKKGHDCN@Can?8t?5get?5string?5at?5?$CF?$CDp?6@ 0000000180006b98     libNonConcreteKlassFilter.obj
 0002:00001bb8       ??_C@_0BP@EKFLGGFJ@Can?8t?5get?5string?5at?5?$CF?$CDp?3?5null?6@ 0000000180006bb8     libNonConcreteKlassFilter.obj
 0002:00001bd8       ??_C@_06ICODBHCL@?5?1?1?5?$CFs@ 0000000180006bd8     libNonConcreteKlassFilter.obj
 0002:00001be0       ??_C@_0DB@KGFPLEGO@?$CIr?5?$DN?5jvmti?9?$DOGetTag?$CIo?0?5?$CGtag?$CJ?$CJ?5?$DN?$DN@ 0000000180006be0     libNonConcreteKlassFilter.obj
 0002:00001c18       ??_C@_0CO@PDAGBCGJ@Can?8t?5GetTag?5for?5object?5?$CFlx?4?5Re@ 0000000180006c18     libNonConcreteKlassFilter.obj
 0002:00001c48       ??_C@_0CH@HPEODOHC@TEST_BUG?3?5Max?4?5number?5of?5refs?5r@ 0000000180006c48     libNonConcreteKlassFilter.obj
 0002:00001c70       ??_C@_0DI@PHFCABIM@?$CIr?5?$DN?5jvmti?9?$DOGetTag?$CIfrom?0?5?$CGtagFr@ 0000000180006c70     libNonConcreteKlassFilter.obj
 0002:00001ca8       ??_C@_0DI@MDEGFNKD@TEST_BUG?3?5Can?8t?5GetTag?5for?5obje@ 0000000180006ca8     libNonConcreteKlassFilter.obj
 0002:00001ce0       ??_C@_0DE@MLELJAHM@?$CIr?5?$DN?5jvmti?9?$DOGetTag?$CIto?0?5?$CGtagTo?$CJ?$CJ@ 0000000180006ce0     libNonConcreteKlassFilter.obj
 0002:00001d20       ??_C@_0JO@KFNGCFDP@jvmtiPrimitiveFieldCallback?5was@ 0000000180006d20     libNonConcreteKlassFilter.obj
 0002:00001dc0       ??_C@_0HC@LHPCIIGP@s?2test?2hotspot?2jtreg?2vmTestbase@ 0000000180006dc0     libNonConcreteKlassFilter.obj
 0002:00001e40       ??_C@_0HO@PLFCBAIO@Unexpected?5value?50x?$CFlX?5was?5repo@ 0000000180006e40     libNonConcreteKlassFilter.obj
 0002:00001ec0       ??_C@_0GI@HJNEEAOA@jvmtiStringPrimitiveValueCallba@ 0000000180006ec0     libNonConcreteKlassFilter.obj
 0002:00001f30       ??_C@_0GH@NICNIGNL@jvmtiArrayPrimitiveValueCallbac@ 0000000180006f30     libNonConcreteKlassFilter.obj
 0002:00001fa0       ??_C@_0KF@CFFNPMEK@jvmtiHeapIterationCallback?5was?5@ 0000000180006fa0     libNonConcreteKlassFilter.obj
 0002:00002048       ??_C@_0BC@BPPEGBIH@Waiting?5debugee?4?6@ 0000000180007048     libNonConcreteKlassFilter.obj
 0002:00002060       ??_C@_0DJ@GDOKODHN@nsk_jvmti_enableEvents?$CIJVMTI_EN@ 0000000180007060     libNonConcreteKlassFilter.obj
 0002:000020a0       ??_C@_0BP@LAIJOMPC@nsk_jvmti_waitForSync?$CItimeout?$CJ@ 00000001800070a0     libNonConcreteKlassFilter.obj
 0002:000020c0       ??_C@_0CO@KMKJIHHP@nullptr?5?$CB?$DN?5?$CIklass?5?$DN?5jni?9?$DOFindCl@ 00000001800070c0     libNonConcreteKlassFilter.obj
 0002:000020f0       ??_C@_0BG@CIAGOPHN@Can?8t?5find?5class?5?$CFs?4?6@ 00000001800070f0     libNonConcreteKlassFilter.obj
 0002:00002108       ??_C@_0DA@ECCIEPML@Iterating?5through?5heap?5with?5kla@ 0000000180007108     libNonConcreteKlassFilter.obj
 0002:00002140       ??_C@_0ED@KPJIJALL@jvmti?9?$DOIterateThroughHeap?$CI0?0?5kl@ 0000000180007140     libNonConcreteKlassFilter.obj
 0002:00002188       ??_C@_0DN@BFFOLECM@Iterating?5through?5heap?5with?5kla@ 0000000180007188     libNonConcreteKlassFilter.obj
 0002:000021c8       ??_C@_0DH@CDNBMDMM@nullptr?5?$CB?$DN?5?$CIklass?5?$DN?5jni?9?$DOFindCl@ 00000001800071c8     libNonConcreteKlassFilter.obj
 0002:00002200       ??_C@_0BA@JJLOPNCP@java?1lang?1Class@ 0000000180007200     libNonConcreteKlassFilter.obj
 0002:00002210       ??_C@_0CD@CMAOCJEE@Can?8t?5find?5class?5java?1lang?1Clas@ 0000000180007210     libNonConcreteKlassFilter.obj
 0002:00002240       ??_C@_0GH@MFPGFGFO@Primitive?5static?5field?5with?5val@ 0000000180007240     libNonConcreteKlassFilter.obj
 0002:000022a8       ??_C@_0BH@LECMGIIA@nsk_jvmti_resumeSync?$CI?$CJ@ 00000001800072a8     libNonConcreteKlassFilter.obj
 0002:000022c0       ??_C@_0BB@CGPOECH@jvmti?5?$CB?$DN?5nullptr@ 00000001800072c0     libNonConcreteKlassFilter.obj
 0002:000022d8       ??_C@_0BO@DBKDIPGD@jvmti?9?$DOAddCapabilities?$CI?$CGcaps?$CJ@ 00000001800072d8     libNonConcreteKlassFilter.obj
 0002:00002300       ??_C@_0EI@OBBECNBE@jvmti?9?$DOSetEventCallbacks?$CI?$CGevent@ 0000000180007300     libNonConcreteKlassFilter.obj
 0002:00002348       ??_C@_0CH@MPLODCED@nsk_jvmti_setAgentProc?$CIagent?0?5n@ 0000000180007348     libNonConcreteKlassFilter.obj
 0002:00002380       ??_C@_1EC@JIJBPKFM@?$AAa?$AAp?$AAi?$AA?9?$AAm?$AAs?$AA?9?$AAw?$AAi?$AAn?$AA?9?$AAc?$AAo?$AAr?$AAe@ 0000000180007380     MSVCRT:thread_safe_statics.obj
 0002:000023c8       ??_C@_1BK@MGMFAEKH@?$AAk?$AAe?$AAr?$AAn?$AAe?$AAl?$AA3?$AA2?$AA?4?$AAd?$AAl?$AAl@ 00000001800073c8     MSVCRT:thread_safe_statics.obj
 0002:000023e8       ??_C@_0BJ@JEBJOJFJ@SleepConditionVariableCS@ 00000001800073e8     MSVCRT:thread_safe_statics.obj
 0002:00002408       ??_C@_0BJ@PGPPEPCC@WakeAllConditionVariable@ 0000000180007408     MSVCRT:thread_safe_statics.obj
 0002:00002428       _pDefaultRawDllMain        0000000180007428     MSVCRT:dll_dllmain.obj
 0002:00002428       _pRawDllMain               0000000180007428     MSVCRT:dll_dllmain.obj
 0002:00002430       __xmm@ffffffffffffffffffffffffffffffff 0000000180007430     MSVCRT:utility.obj
 0002:00002440       _load_config_used          0000000180007440     MSVCRT:loadcfg.obj
 0002:00002600       _tls_used                  0000000180007600     MSVCRT:tlssup.obj
 0002:00002628       __volatile_metadata        0000000180007628     <linker-defined>
 0002:00002a08       __rtc_iaa                  0000000180007a08     MSVCRT:initsect.obj
 0002:00002a10       __rtc_izz                  0000000180007a10     MSVCRT:initsect.obj
 0002:00002a18       __rtc_taa                  0000000180007a18     MSVCRT:initsect.obj
 0002:00002a20       __rtc_tzz                  0000000180007a20     MSVCRT:initsect.obj
 0002:00002a28       _tls_start                 0000000180007a28     MSVCRT:tlssup.obj
 0002:00002a2c       _Init_thread_epoch         0000000180007a2c     MSVCRT:thread_safe_statics.obj
 0002:00002a30       _tls_end                   0000000180007a30     MSVCRT:tlssup.obj
 0002:00003110       __IMPORT_DESCRIPTOR_KERNEL32 0000000180008110     kernel32:KERNEL32.dll
 0002:00003124       __IMPORT_DESCRIPTOR_VCRUNTIME140 0000000180008124     vcruntime:VCRUNTIME140.dll
 0002:00003138       __IMPORT_DESCRIPTOR_api-ms-win-crt-heap-l1-1-0 0000000180008138     ucrt:api-ms-win-crt-heap-l1-1-0.dll
 0002:0000314c       __IMPORT_DESCRIPTOR_api-ms-win-crt-runtime-l1-1-0 000000018000814c     ucrt:api-ms-win-crt-runtime-l1-1-0.dll
 0002:00003160       __IMPORT_DESCRIPTOR_api-ms-win-crt-convert-l1-1-0 0000000180008160     ucrt:api-ms-win-crt-convert-l1-1-0.dll
 0002:00003174       __IMPORT_DESCRIPTOR_api-ms-win-crt-stdio-l1-1-0 0000000180008174     ucrt:api-ms-win-crt-stdio-l1-1-0.dll
 0002:00003188       __IMPORT_DESCRIPTOR_api-ms-win-crt-string-l1-1-0 0000000180008188     ucrt:api-ms-win-crt-string-l1-1-0.dll
 0002:0000319c       __NULL_IMPORT_DESCRIPTOR   000000018000819c     kernel32:KERNEL32.dll
 0003:00000050       _Init_global_epoch         0000000180009050     MSVCRT:thread_safe_statics.obj
 0003:00000060       __security_cookie          0000000180009060     MSVCRT:gs_cookie.obj
 0003:00000068       __security_cookie_complement 0000000180009068     MSVCRT:gs_cookie.obj
 0003:00000070       __scrt_native_dllmain_reason 0000000180009070     MSVCRT:utility.obj
 0003:00000078       __isa_available            0000000180009078     MSVCRT:cpu_disp.obj
 0003:0000007c       __isa_enabled              000000018000907c     MSVCRT:cpu_disp.obj
 0003:00000080       __memset_fast_string_threshold 0000000180009080     MSVCRT:cpu_disp.obj
 0003:00000088       __memset_nt_threshold      0000000180009088     MSVCRT:cpu_disp.obj
 0003:00000090       __scrt_ucrt_dll_is_in_use  0000000180009090     MSVCRT:ucrt_stubs.obj
 0003:000000a0       g_wrongHeapCallbacks       00000001800090a0     libNonConcreteKlassFilter.obj
 0003:00000120       g_szTagInfo                0000000180009120     libNonConcreteKlassFilter.obj
 0003:00002060       g_tagFlags                 000000018000b060     libNonConcreteKlassFilter.obj
 0003:00002448       g_refsToVerifyCnt          000000018000b448     libNonConcreteKlassFilter.obj
 0003:0000244c       g_fakeUserData             000000018000b44c     libNonConcreteKlassFilter.obj
 0003:00002450       g_tagVisitCount            000000018000b450     libNonConcreteKlassFilter.obj
 0003:000033f0       g_refsToVerify             000000018000c3f0     libNonConcreteKlassFilter.obj
 0003:0001aaf0       g_userDataError            0000000180023af0     libNonConcreteKlassFilter.obj
 0003:0001ac98       ?_OptionsStorage@?1??__local_stdio_printf_options@@9@4_KA 0000000180023c98     libNonConcreteKlassFilter.obj
 0003:0001b258       _tls_index                 0000000180024258     MSVCRT:tlssup.obj
 0003:0001b260       __scrt_current_native_startup_state 0000000180024260     MSVCRT:utility.obj
 0003:0001b268       __scrt_native_startup_lock 0000000180024268     MSVCRT:utility.obj
 0003:0001b2a8       __scrt_debugger_hook_flag  00000001800242a8     MSVCRT:utility_desktop.obj
 0003:0001b2b0       ?__type_info_root_node@@3U__type_info_node@@A 00000001800242b0     MSVCRT:tncleanup.obj
 0003:0001b2c0       ?_OptionsStorage@?1??__local_stdio_scanf_options@@9@4_KA 00000001800242c0     MSVCRT:default_local_stdio_options.obj
 0003:0001b2c8       __favor                    00000001800242c8     MSVCRT:cpu_disp.obj
 0003:0001b2d0       __dyn_tls_init_callback    00000001800242d0     <common>

 entry point at        0001:00003010

 Static symbols

 0000:fffd9000       .debug$S                   0000000180000000     NonConcreteKlassFilter.exp
 0000:fffd9000       .debug$S                   0000000180000000     vcruntime:VCRUNTIME140.dll
 0000:fffd9000       .debug$S                   0000000180000000     vcruntime:VCRUNTIME140.dll
 0000:fffd9000       .debug$S                   0000000180000000     vcruntime:VCRUNTIME140.dll
 0000:fffd9000       .debug$S                   0000000180000000     vcruntime:VCRUNTIME140.dll
 0000:fffd9000       .debug$S                   0000000180000000     vcruntime:VCRUNTIME140.dll
 0000:fffd9000       .debug$S                   0000000180000000     vcruntime:VCRUNTIME140.dll
 0000:fffd9000       .debug$S                   0000000180000000     vcruntime:VCRUNTIME140.dll
 0000:fffd9000       .debug$S                   0000000180000000     ucrt:api-ms-win-crt-convert-l1-1-0.dll
 0000:fffd9000       .debug$S                   0000000180000000     ucrt:api-ms-win-crt-heap-l1-1-0.dll
 0000:fffd9000       .debug$S                   0000000180000000     ucrt:api-ms-win-crt-heap-l1-1-0.dll
 0000:fffd9000       .debug$S                   0000000180000000     ucrt:api-ms-win-crt-heap-l1-1-0.dll
 0000:fffd9000       .debug$S                   0000000180000000     ucrt:api-ms-win-crt-heap-l1-1-0.dll
 0000:fffd9000       .debug$S                   0000000180000000     ucrt:api-ms-win-crt-runtime-l1-1-0.dll
 0000:fffd9000       .debug$S                   0000000180000000     ucrt:api-ms-win-crt-runtime-l1-1-0.dll
 0000:fffd9000       .debug$S                   0000000180000000     ucrt:api-ms-win-crt-runtime-l1-1-0.dll
 0000:fffd9000       .debug$S                   0000000180000000     ucrt:api-ms-win-crt-runtime-l1-1-0.dll
 0000:fffd9000       .debug$S                   0000000180000000     ucrt:api-ms-win-crt-runtime-l1-1-0.dll
 0000:fffd9000       .debug$S                   0000000180000000     ucrt:api-ms-win-crt-runtime-l1-1-0.dll
 0000:fffd9000       .debug$S                   0000000180000000     ucrt:api-ms-win-crt-runtime-l1-1-0.dll
 0000:fffd9000       .debug$S                   0000000180000000     ucrt:api-ms-win-crt-runtime-l1-1-0.dll
 0000:fffd9000       .debug$S                   0000000180000000     ucrt:api-ms-win-crt-runtime-l1-1-0.dll
 0000:fffd9000       .debug$S                   0000000180000000     ucrt:api-ms-win-crt-runtime-l1-1-0.dll
 0000:fffd9000       .debug$S                   0000000180000000     ucrt:api-ms-win-crt-runtime-l1-1-0.dll
 0000:fffd9000       .debug$S                   0000000180000000     ucrt:api-ms-win-crt-runtime-l1-1-0.dll
 0000:fffd9000       .debug$S                   0000000180000000     ucrt:api-ms-win-crt-runtime-l1-1-0.dll
 0000:fffd9000       .debug$S                   0000000180000000     ucrt:api-ms-win-crt-runtime-l1-1-0.dll
 0000:fffd9000       .debug$S                   0000000180000000     ucrt:api-ms-win-crt-runtime-l1-1-0.dll
 0000:fffd9000       .debug$S                   0000000180000000     ucrt:api-ms-win-crt-runtime-l1-1-0.dll
 0000:fffd9000       .debug$S                   0000000180000000     ucrt:api-ms-win-crt-stdio-l1-1-0.dll
 0000:fffd9000       .debug$S                   0000000180000000     ucrt:api-ms-win-crt-stdio-l1-1-0.dll
 0000:fffd9000       .debug$S                   0000000180000000     ucrt:api-ms-win-crt-stdio-l1-1-0.dll
 0000:fffd9000       .debug$S                   0000000180000000     ucrt:api-ms-win-crt-stdio-l1-1-0.dll
 0000:fffd9000       .debug$S                   0000000180000000     ucrt:api-ms-win-crt-stdio-l1-1-0.dll
 0000:fffd9000       .debug$S                   0000000180000000     ucrt:api-ms-win-crt-stdio-l1-1-0.dll
 0000:fffd9000       .debug$S                   0000000180000000     ucrt:api-ms-win-crt-stdio-l1-1-0.dll
 0000:fffd9000       .debug$S                   0000000180000000     ucrt:api-ms-win-crt-stdio-l1-1-0.dll
 0000:fffd9000       .debug$S                   0000000180000000     ucrt:api-ms-win-crt-stdio-l1-1-0.dll
 0000:fffd9000       .debug$S                   0000000180000000     ucrt:api-ms-win-crt-stdio-l1-1-0.dll
 0000:fffd9000       .debug$S                   0000000180000000     ucrt:api-ms-win-crt-string-l1-1-0.dll
 0000:fffd9000       .debug$S                   0000000180000000     ucrt:api-ms-win-crt-string-l1-1-0.dll
 0000:fffd9000       .debug$S                   0000000180000000     ucrt:api-ms-win-crt-string-l1-1-0.dll
 0000:fffd9000       .debug$S                   0000000180000000     ucrt:api-ms-win-crt-string-l1-1-0.dll
 0000:fffd9000       .debug$S                   0000000180000000     ucrt:api-ms-win-crt-string-l1-1-0.dll
 0000:fffd9000       .debug$S                   0000000180000000     ucrt:api-ms-win-crt-string-l1-1-0.dll
 0000:fffd9000       .debug$S                   0000000180000000     ucrt:api-ms-win-crt-string-l1-1-0.dll
 0000:fffd9000       .debug$S                   0000000180000000     ucrt:api-ms-win-crt-string-l1-1-0.dll
 0000:fffd9000       .debug$S                   0000000180000000     kernel32:KERNEL32.dll
 0000:fffd9000       .debug$S                   0000000180000000     kernel32:KERNEL32.dll
 0000:fffd9000       .debug$S                   0000000180000000     kernel32:KERNEL32.dll
 0000:fffd9000       .debug$S                   0000000180000000     kernel32:KERNEL32.dll
 0000:fffd9000       .debug$S                   0000000180000000     kernel32:KERNEL32.dll
 0000:fffd9000       .debug$S                   0000000180000000     kernel32:KERNEL32.dll
 0000:fffd9000       .debug$S                   0000000180000000     kernel32:KERNEL32.dll
 0000:fffd9000       .debug$S                   0000000180000000     kernel32:KERNEL32.dll
 0000:fffd9000       .debug$S                   0000000180000000     kernel32:KERNEL32.dll
 0000:fffd9000       .debug$S                   0000000180000000     kernel32:KERNEL32.dll
 0000:fffd9000       .debug$S                   0000000180000000     kernel32:KERNEL32.dll
 0000:fffd9000       .debug$S                   0000000180000000     kernel32:KERNEL32.dll
 0000:fffd9000       .debug$S                   0000000180000000     kernel32:KERNEL32.dll
 0000:fffd9000       .debug$S                   0000000180000000     kernel32:KERNEL32.dll
 0000:fffd9000       .debug$S                   0000000180000000     kernel32:KERNEL32.dll
 0000:fffd9000       .debug$S                   0000000180000000     kernel32:KERNEL32.dll
 0000:fffd9000       .debug$S                   0000000180000000     kernel32:KERNEL32.dll
 0000:fffd9000       .debug$S                   0000000180000000     kernel32:KERNEL32.dll
 0000:fffd9000       .debug$S                   0000000180000000     kernel32:KERNEL32.dll
 0000:fffd9000       .debug$S                   0000000180000000     kernel32:KERNEL32.dll
 0000:fffd9000       .debug$S                   0000000180000000     kernel32:KERNEL32.dll
 0000:fffd9000       .debug$S                   0000000180000000     kernel32:KERNEL32.dll
 0000:fffd9000       .debug$S                   0000000180000000     kernel32:KERNEL32.dll
 0000:fffd9000       .debug$S                   0000000180000000     kernel32:KERNEL32.dll
 0000:fffd9000       .debug$S                   0000000180000000     kernel32:KERNEL32.dll
 0000:fffd9000       .debug$S                   0000000180000000     kernel32:KERNEL32.dll
 0000:fffd9000       .debug$S                   0000000180000000     kernel32:KERNEL32.dll
 0000:fffd9000       .debug$S                   0000000180000000     kernel32:KERNEL32.dll
 0001:00000e8c       addRefToVerify             0000000180001e8c f   libNonConcreteKlassFilter.obj
 0001:00000ef8       agent                      0000000180001ef8 f   libNonConcreteKlassFilter.obj
 0001:00001348       agentThreadWrapper         0000000180002348 f   libNonConcreteKlassFilter.obj
 0001:000014e4       check_option               00000001800024e4 f   libNonConcreteKlassFilter.obj
 0001:000017e8       file_basename              00000001800027e8 f   libNonConcreteKlassFilter.obj
 0001:000024c0       startAgentThreadWrapper    00000001800034c0 f   libNonConcreteKlassFilter.obj
 0001:00002830       syncDebuggeeStatus         0000000180003830 f   libNonConcreteKlassFilter.obj
 0001:00002ad0       capture_previous_context   0000000180003ad0 f   MSVCRT:gs_report.obj
 0001:00002b44       ?__scrt_initialize_thread_safe_statics@@YAHXZ 0000000180003b44 f   MSVCRT:thread_safe_statics.obj
 0001:00002c14       ?__scrt_uninitialize_thread_safe_statics@@YAXXZ 0000000180003c14 f   MSVCRT:thread_safe_statics.obj
 0001:00002cc0       $$000000                   0000000180003cc0     MSVCRT:amdsecgs.obj
 0001:00002cf0       ?dllmain_crt_dispatch@@YAHQEAUHINSTANCE__@@KQEAX@Z 0000000180003cf0 f   MSVCRT:dll_dllmain.obj
 0001:00002d40       ?dllmain_crt_process_attach@@YAHQEAUHINSTANCE__@@QEAX@Z 0000000180003d40 f   MSVCRT:dll_dllmain.obj
 0001:00002e58       ?dllmain_crt_process_detach@@YAH_N@Z 0000000180003e58 f   MSVCRT:dll_dllmain.obj
 0001:00002edc       ?dllmain_dispatch@@YAHQEAUHINSTANCE__@@KQEAX@Z 0000000180003edc f   MSVCRT:dll_dllmain.obj
 0001:000038f0       $$000000                   00000001800048f0     MSVCRT:guard_dispatch.obj
 0001:00003910       $$000000                   0000000180004910     MSVCRT:guard_xfg_dispatch.obj
 0001:00003926       ?fin$0@?0??dllmain_crt_process_attach@@YAHQEAUHINSTANCE__@@QEAX@Z@4HA 0000000180004926 f   MSVCRT:dll_dllmain.obj
 0001:0000393d       ?fin$0@?0??dllmain_crt_process_detach@@YAH_N@Z@4HA 000000018000493d f   MSVCRT:dll_dllmain.obj
 0001:00003956       ?fin$1@?0??dllmain_crt_process_detach@@YAH_N@Z@4HA 0000000180004956 f   MSVCRT:dll_dllmain.obj
 0001:0000396a       ?filt$0@?0??dllmain_dispatch@@YAHQEAUHINSTANCE__@@KQEAX@Z@4HA 000000018000496a f   MSVCRT:dll_dllmain.obj
 0001:000039a0       __scrt_is_nonwritable_in_current_image$filt$0 00000001800049a0 f   MSVCRT:utility.obj
 0002:00000218       ?__scrt_initialize_tss_var@@3P6AHXZEA 0000000180005218     MSVCRT:thread_safe_statics.obj
 0002:00000340       ?opcLengths@@3QBEB         0000000180005340     libNonConcreteKlassFilter.obj
 0002:00002370       GS_ExceptionPointers       0000000180007370     MSVCRT:gs_report.obj
 0002:00002a38       $unwind$fprintf            0000000180007a38     libNonConcreteKlassFilter.obj
 0002:00002a44       $unwind$printf             0000000180007a44     libNonConcreteKlassFilter.obj
 0002:00002a50       $unwind$?NewObject@JNIEnv_@@QEAAPEAV_jobject@@PEAV_jclass@@PEAU_jmethodID@@ZZ 0000000180007a50     libNonConcreteKlassFilter.obj
 0002:00002a50       $unwind$nsk_lcomplain      0000000180007a50     libNonConcreteKlassFilter.obj
 0002:00002a50       $unwind$nsk_ldisplay       0000000180007a50     libNonConcreteKlassFilter.obj
 0002:00002a58       $unwind$nsk_jvmti_waitForSync 0000000180007a58     libNonConcreteKlassFilter.obj
 0002:00002a58       $unwind$nsk_lvdisplay      0000000180007a58     libNonConcreteKlassFilter.obj
 0002:00002a58       $unwind$_RTC_Initialize    0000000180007a58     MSVCRT:initsect.obj
 0002:00002a58       $unwind$_RTC_Terminate     0000000180007a58     MSVCRT:initsect.obj
 0002:00002a58       $unwind$?__scrt_initialize_thread_safe_statics@@YAHXZ 0000000180007a58     MSVCRT:thread_safe_statics.obj
 0002:00002a64       $unwind$nsk_complain       0000000180007a64     libNonConcreteKlassFilter.obj
 0002:00002a64       $unwind$nsk_printf         0000000180007a64     libNonConcreteKlassFilter.obj
 0002:00002a6c       $unwind$nsk_lvcomplain     0000000180007a6c     libNonConcreteKlassFilter.obj
 0002:00002a84       $unwind$nsk_ltrace         0000000180007a84     libNonConcreteKlassFilter.obj
 0002:00002a84       $unwind$__report_gsfailure 0000000180007a84     MSVCRT:gs_report.obj
 0002:00002a8c       $unwind$nsk_lvtrace        0000000180007a8c     libNonConcreteKlassFilter.obj
 0002:00002a8c       $unwind$__raise_securityfailure 0000000180007a8c     MSVCRT:gs_report.obj
 0002:00002a8c       $unwind$__scrt_initialize_crt 0000000180007a8c     MSVCRT:utility.obj
 0002:00002a8c       $unwind$__scrt_initialize_onexit_tables 0000000180007a8c     MSVCRT:utility.obj
 0002:00002a8c       $unwind$__scrt_release_startup_lock 0000000180007a8c     MSVCRT:utility.obj
 0002:00002a8c       $unwind$__scrt_uninitialize_crt 0000000180007a8c     MSVCRT:utility.obj
 0002:00002a8c       $unwind$_onexit            0000000180007a8c     MSVCRT:utility.obj
 0002:00002a94       $unwind$nsk_lverify        0000000180007a94     libNonConcreteKlassFilter.obj
 0002:00002aa4       $unwind$nsk_vprintf        0000000180007aa4     libNonConcreteKlassFilter.obj
 0002:00002ab4       $unwind$?nsk_jni_lverify@@YAHHPEAUJNIEnv_@@HQEBDH1ZZ 0000000180007ab4     libNonConcreteKlassFilter.obj
 0002:00002ac8       $unwind$?nsk_jni_check_exception@@YAHPEAUJNIEnv_@@QEBDH@Z 0000000180007ac8     libNonConcreteKlassFilter.obj
 0002:00002ae4       $unwind$nsk_jvmti_parseOptions 0000000180007ae4     libNonConcreteKlassFilter.obj
 0002:00002b00       $unwind$nsk_jvmti_createJVMTIEnv 0000000180007b00     libNonConcreteKlassFilter.obj
 0002:00002b14       $unwind$Java_nsk_jvmti_unit_FollowReferences_FollowRefObjects_resetTags 0000000180007b14     libNonConcreteKlassFilter.obj
 0002:00002b14       $unwind$addRefToVerify     0000000180007b14     libNonConcreteKlassFilter.obj
 0002:00002b14       $unwind$nsk_jvmti_resetAgentData 0000000180007b14     libNonConcreteKlassFilter.obj
 0002:00002b14       $unwind$nsk_jvmti_resumeSync 0000000180007b14     libNonConcreteKlassFilter.obj
 0002:00002b14       $unwind$nsk_jvmti_setFailStatus 0000000180007b14     libNonConcreteKlassFilter.obj
 0002:00002b14       $unwind$__scrt_initialize_default_local_stdio_options 0000000180007b14     MSVCRT:default_local_stdio_options.obj
 0002:00002b14       $unwind$?dllmain_crt_dispatch@@YAHQEAUHINSTANCE__@@KQEAX@Z 0000000180007b14     MSVCRT:dll_dllmain.obj
 0002:00002b14       $unwind$DllMain            0000000180007b14     MSVCRT:dll_dllmain_stub.obj
 0002:00002b14       $unwind$__GSHandlerCheck   0000000180007b14     MSVCRT:gshandler.obj
 0002:00002b14       $unwind$?__scrt_uninitialize_thread_safe_statics@@YAXXZ 0000000180007b14     MSVCRT:thread_safe_statics.obj
 0002:00002b14       $unwind$__scrt_acquire_startup_lock 0000000180007b14     MSVCRT:utility.obj
 0002:00002b14       $unwind$__scrt_dllmain_after_initialize_c 0000000180007b14     MSVCRT:utility.obj
 0002:00002b14       $unwind$__scrt_dllmain_before_initialize_c 0000000180007b14     MSVCRT:utility.obj
 0002:00002b14       $unwind$__scrt_dllmain_crt_thread_attach 0000000180007b14     MSVCRT:utility.obj
 0002:00002b14       $unwind$__scrt_dllmain_crt_thread_detach 0000000180007b14     MSVCRT:utility.obj
 0002:00002b14       $unwind$__scrt_dllmain_uninitialize_c 0000000180007b14     MSVCRT:utility.obj
 0002:00002b14       $unwind$__scrt_dllmain_uninitialize_critical 0000000180007b14     MSVCRT:utility.obj
 0002:00002b14       $unwind$atexit             0000000180007b14     MSVCRT:utility.obj
 0002:00002b1c       $unwind$nsk_jvmti_enableEvents 0000000180007b1c     libNonConcreteKlassFilter.obj
 0002:00002b34       $unwind$nsk_jvmti_lverify  0000000180007b34     libNonConcreteKlassFilter.obj
 0002:00002b48       $unwind$exitOnError        0000000180007b48     libNonConcreteKlassFilter.obj
 0002:00002b58       $unwind$check_option       0000000180007b58     libNonConcreteKlassFilter.obj
 0002:00002b58       $unwind$_DllMainCRTStartup 0000000180007b58     MSVCRT:dll_dllmain.obj
 0002:00002b68       $unwind$Java_nsk_share_jvmti_ArgumentHandler_getAgentOptionsString 0000000180007b68     libNonConcreteKlassFilter.obj
 0002:00002b7c       $unwind$Java_nsk_jvmti_unit_FollowReferences_FollowRefObjects_getTag 0000000180007b7c     libNonConcreteKlassFilter.obj
 0002:00002b7c       $unwind$Java_nsk_share_jvmti_DebugeeClass_checkStatus 0000000180007b7c     libNonConcreteKlassFilter.obj
 0002:00002b7c       $unwind$agentThreadWrapper 0000000180007b7c     libNonConcreteKlassFilter.obj
 0002:00002b8c       $unwind$startAgentThreadWrapper 0000000180007b8c     libNonConcreteKlassFilter.obj
 0002:00002ba8       $unwind$syncDebuggeeStatus 0000000180007ba8     libNonConcreteKlassFilter.obj
 0002:00002ba8       $unwind$__scrt_dllmain_exception_filter 0000000180007ba8     MSVCRT:utility.obj
 0002:00002bbc       $unwind$Java_nsk_share_jvmti_DebugeeClass_resetAgentData 0000000180007bbc     libNonConcreteKlassFilter.obj
 0002:00002bc4       $unwind$MA_checkStatus     0000000180007bc4     libNonConcreteKlassFilter.obj
 0002:00002bd8       $unwind$Java_nsk_jvmti_unit_FollowReferences_FollowRefObjects_setTag 0000000180007bd8     libNonConcreteKlassFilter.obj
 0002:00002bf0       $unwind$Java_nsk_jvmti_unit_FollowReferences_FollowRefObjects_addRefToVerify 0000000180007bf0     libNonConcreteKlassFilter.obj
 0002:00002c0c       $unwind$Agent_Initialize   0000000180007c0c     libNonConcreteKlassFilter.obj
 0002:00002c2c       $unwind$array_callback     0000000180007c2c     libNonConcreteKlassFilter.obj
 0002:00002c2c       $unwind$field_callback     0000000180007c2c     libNonConcreteKlassFilter.obj
 0002:00002c2c       $unwind$heap_callback      0000000180007c2c     libNonConcreteKlassFilter.obj
 0002:00002c2c       $unwind$string_callback    0000000180007c2c     libNonConcreteKlassFilter.obj
 0002:00002c34       $unwind$agent              0000000180007c34     libNonConcreteKlassFilter.obj
 0002:00002c54       $unwind$capture_previous_context 0000000180007c54     MSVCRT:gs_report.obj
 0002:00002c60       $unwind$__GSHandlerCheckCommon 0000000180007c60     MSVCRT:gshandler.obj
 0002:00002c68       $xdatasym                  0000000180007c68     MSVCRT:amdsecgs.obj
 0002:00002c6c       $unwind$?dllmain_crt_process_attach@@YAHQEAUHINSTANCE__@@QEAX@Z 0000000180007c6c     MSVCRT:dll_dllmain.obj
 0002:00002ca8       $unwind$?fin$0@?0??dllmain_crt_process_attach@@YAHQEAUHINSTANCE__@@QEAX@Z@4HA 0000000180007ca8     MSVCRT:dll_dllmain.obj
 0002:00002ca8       $unwind$?fin$0@?0??dllmain_crt_process_detach@@YAH_N@Z@4HA 0000000180007ca8     MSVCRT:dll_dllmain.obj
 0002:00002ca8       $unwind$?fin$1@?0??dllmain_crt_process_detach@@YAH_N@Z@4HA 0000000180007ca8     MSVCRT:dll_dllmain.obj
 0002:00002cb0       $unwind$?dllmain_crt_process_detach@@YAH_N@Z 0000000180007cb0     MSVCRT:dll_dllmain.obj
 0002:00002d04       $unwind$?dllmain_dispatch@@YAHQEAUHINSTANCE__@@KQEAX@Z 0000000180007d04     MSVCRT:dll_dllmain.obj
 0002:00002d2c       $unwind$?filt$0@?0??dllmain_dispatch@@YAHQEAUHINSTANCE__@@KQEAX@Z@4HA 0000000180007d2c     MSVCRT:dll_dllmain.obj
 0002:00002d34       $unwind$__scrt_is_nonwritable_in_current_image 0000000180007d34     MSVCRT:utility.obj
 0002:00002d54       $unwind$__scrt_is_nonwritable_in_current_image$filt$0 0000000180007d54     MSVCRT:utility.obj
 0002:00002d5c       $unwind$__scrt_fastfail    0000000180007d5c     MSVCRT:utility_desktop.obj
 0002:00002d6c       $unwind$__security_init_cookie 0000000180007d6c     MSVCRT:gs_support.obj
 0002:00002d78       $unwind$__isa_available_init 0000000180007d78     MSVCRT:cpu_disp.obj
 0002:00002d88       $xdatasym                  0000000180007d88     MSVCRT:guard_dispatch.obj
 0002:00002d90       $xdatasym                  0000000180007d90     MSVCRT:guard_xfg_dispatch.obj
 0002:00002da0       .edata                     0000000180007da0     NonConcreteKlassFilter.exp
 0002:00002dc8       rgpv                       0000000180007dc8     NonConcreteKlassFilter.exp
 0002:00002e00       rgszName                   0000000180007e00     NonConcreteKlassFilter.exp
 0002:00002e38       rgwOrd                     0000000180007e38     NonConcreteKlassFilter.exp
 0002:00002e54       szName                     0000000180007e54     NonConcreteKlassFilter.exp
 0002:00002e6f       $N00001                    0000000180007e6f     NonConcreteKlassFilter.exp
 0002:00002e7e       $N00002                    0000000180007e7e     NonConcreteKlassFilter.exp
 0002:00002e8b       $N00003                    0000000180007e8b     NonConcreteKlassFilter.exp
 0002:00002ed0       $N00004                    0000000180007ed0     NonConcreteKlassFilter.exp
 0002:00002f0d       $N00005                    0000000180007f0d     NonConcreteKlassFilter.exp
 0002:00002f55       $N00006                    0000000180007f55     NonConcreteKlassFilter.exp
 0002:00002f95       $N00007                    0000000180007f95     NonConcreteKlassFilter.exp
 0002:00002fd2       $N00008                    0000000180007fd2     NonConcreteKlassFilter.exp
 0002:0000300d       $N00009                    000000018000800d     NonConcreteKlassFilter.exp
 0002:0000303b       $N00010                    000000018000803b     NonConcreteKlassFilter.exp
 0002:0000306c       $N00011                    000000018000806c     NonConcreteKlassFilter.exp
 0002:0000309b       $N00012                    000000018000809b     NonConcreteKlassFilter.exp
 0002:000030ca       $N00013                    00000001800080ca     NonConcreteKlassFilter.exp
 0002:000030ff       $N00014                    00000001800080ff     NonConcreteKlassFilter.exp
 0002:00003562       .idata$6                   0000000180008562     kernel32:KERNEL32.dll
 0002:000035c6       .idata$6                   00000001800085c6     vcruntime:VCRUNTIME140.dll
 0002:00003758       .idata$6                   0000000180008758     ucrt:api-ms-win-crt-heap-l1-1-0.dll
 0002:00003778       .idata$6                   0000000180008778     ucrt:api-ms-win-crt-runtime-l1-1-0.dll
 0002:0000379a       .idata$6                   000000018000879a     ucrt:api-ms-win-crt-convert-l1-1-0.dll
 0002:000037bc       .idata$6                   00000001800087bc     ucrt:api-ms-win-crt-stdio-l1-1-0.dll
 0002:000037dc       .idata$6                   00000001800087dc     ucrt:api-ms-win-crt-string-l1-1-0.dll
 0003:00000000       ?codeAttributeName@@3PEBDEB 0000000180009000     libNonConcreteKlassFilter.obj
 0003:00000008       ?lineNumberAttributeName@@3PEBDEB 0000000180009008     libNonConcreteKlassFilter.obj
 0003:00000010       ?localVarAttributeName@@3PEBDEB 0000000180009010     libNonConcreteKlassFilter.obj
 0003:00000018       ?localVarTypeAttributeName@@3PEBDEB 0000000180009018     libNonConcreteKlassFilter.obj
 0003:00000020       ?stackMapAttributeName@@3PEBDEB 0000000180009020     libNonConcreteKlassFilter.obj
 0003:00000028       ?callBytes@@3PAEA          0000000180009028     libNonConcreteKlassFilter.obj
 0003:0000002c       ?allocBytes@@3PAEA         000000018000902c     libNonConcreteKlassFilter.obj
 0003:00000030       expected_values            0000000180009030     libNonConcreteKlassFilter.obj
 0003:00000040       types                      0000000180009040     libNonConcreteKlassFilter.obj
 0003:0001aaf4       redefineAttempted          0000000180023af4     libNonConcreteKlassFilter.obj
 0003:0001aaf8       nsk_context                0000000180023af8     libNonConcreteKlassFilter.obj
 0003:0001ab04       redefineSucceed            0000000180023b04     libNonConcreteKlassFilter.obj
 0003:0001ab08       agentFailed                0000000180023b08     libNonConcreteKlassFilter.obj
 0003:0001ab0c       currentAgentStatus         0000000180023b0c     libNonConcreteKlassFilter.obj
 0003:0001ab10       context                    0000000180023b10     libNonConcreteKlassFilter.obj
 0003:0001abc8       agentThread                0000000180023bc8     libNonConcreteKlassFilter.obj
 0003:0001abd0       agentThreadProc            0000000180023bd0     libNonConcreteKlassFilter.obj
 0003:0001abd8       agentThreadArg             0000000180023bd8     libNonConcreteKlassFilter.obj
 0003:0001abe0       agent_data                 0000000180023be0     libNonConcreteKlassFilter.obj
 0003:0001abf0       jvmti_env                  0000000180023bf0     libNonConcreteKlassFilter.obj
 0003:0001abf8       jvm                        0000000180023bf8     libNonConcreteKlassFilter.obj
 0003:0001ac00       jni_env                    0000000180023c00     libNonConcreteKlassFilter.obj
 0003:0001ac08       checkStatus_func           0000000180023c08     libNonConcreteKlassFilter.obj
 0003:0001ac10       ?codeAttributeIndex@@3GA   0000000180023c10     libNonConcreteKlassFilter.obj
 0003:0001ac14       ?lineNumberAttributeIndex@@3GA 0000000180023c14     libNonConcreteKlassFilter.obj
 0003:0001ac18       ?localVarAttributeIndex@@3GA 0000000180023c18     libNonConcreteKlassFilter.obj
 0003:0001ac1c       ?localVarTypeAttributeIndex@@3GA 0000000180023c1c     libNonConcreteKlassFilter.obj
 0003:0001ac20       ?stackMapAttributeIndex@@3GA 0000000180023c20     libNonConcreteKlassFilter.obj
 0003:0001ac24       ?stackFrameOffset@@3GA     0000000180023c24     libNonConcreteKlassFilter.obj
 0003:0001ac28       ?mode@@3HA                 0000000180023c28     libNonConcreteKlassFilter.obj
 0003:0001ac2c       ?constantPoolSize@@3GA     0000000180023c2c     libNonConcreteKlassFilter.obj
 0003:0001ac30       ?orig@@3PEBEEB             0000000180023c30     libNonConcreteKlassFilter.obj
 0003:0001ac38       ?gen@@3PEAEEA              0000000180023c38     libNonConcreteKlassFilter.obj
 0003:0001ac40       ?inputPos@@3PEAEEA         0000000180023c40     libNonConcreteKlassFilter.obj
 0003:0001ac48       ?endPos@@3PEBEEB           0000000180023c48     libNonConcreteKlassFilter.obj
 0003:0001ac50       ?genPos@@3PEAEEA           0000000180023c50     libNonConcreteKlassFilter.obj
 0003:0001ac58       ?markPos@@3PEAEEA          0000000180023c58     libNonConcreteKlassFilter.obj
 0003:0001ac60       ?constantPool@@3PEAPEADEA  0000000180023c60     libNonConcreteKlassFilter.obj
 0003:0001ac68       ?constantPoolCount@@3GA    0000000180023c68     libNonConcreteKlassFilter.obj
 0003:0001ac6c       ?zeroBytes@@3PAEA          0000000180023c6c     libNonConcreteKlassFilter.obj
 0003:0001ac70       ?codeLength@@3IA           0000000180023c70     libNonConcreteKlassFilter.obj
 0003:0001ac74       phase                      0000000180023c74     libNonConcreteKlassFilter.obj
 0003:0001ac78       ?map@@3PEAIEA              0000000180023c78     libNonConcreteKlassFilter.obj
 0003:0001ac80       ?widening@@3PEACEA         0000000180023c80     libNonConcreteKlassFilter.obj
 0003:0001ac88       occurancies                0000000180023c88     libNonConcreteKlassFilter.obj
 0003:0001ac90       timeout                    0000000180023c90     libNonConcreteKlassFilter.obj
 0003:0001aca0       GS_ExceptionRecord         0000000180023ca0     MSVCRT:gs_report.obj
 0003:0001ad40       GS_ContextRecord           0000000180023d40     MSVCRT:gs_report.obj
 0003:0001b210       ?g_tss_cv@@3U_RTL_CONDITION_VARIABLE@@A 0000000180024210     MSVCRT:thread_safe_statics.obj
 0003:0001b218       ?g_tss_event@@3PEAXEA      0000000180024218     MSVCRT:thread_safe_statics.obj
 0003:0001b220       ?g_tss_mutex@@3U_RTL_CRITICAL_SECTION@@A 0000000180024220     MSVCRT:thread_safe_statics.obj
 0003:0001b248       ?g_sleep_condition_variable_cs@@3P6AHPEAU_RTL_CONDITION_VARIABLE@@PEAU_RTL_CRITICAL_SECTION@@K@ZEA 0000000180024248     MSVCRT:thread_safe_statics.obj
 0003:0001b250       ?g_wake_all_condition_variable@@3P6AXPEAU_RTL_CONDITION_VARIABLE@@@ZEA 0000000180024250     MSVCRT:thread_safe_statics.obj
 0003:0001b25c       ?__proc_attached@@3HA      000000018002425c     MSVCRT:dll_dllmain.obj
 0003:0001b270       ?is_initialized_as_dll@@3_NA 0000000180024270     MSVCRT:utility.obj
 0003:0001b271       ?module_local_atexit_table_initialized@@3_NA 0000000180024271     MSVCRT:utility.obj
 0003:0001b278       ?module_local_atexit_table@@3U_onexit_table_t@@A 0000000180024278     MSVCRT:utility.obj
 0003:0001b290       ?module_local_at_quick_exit_table@@3U_onexit_table_t@@A 0000000180024290     MSVCRT:utility.obj
